:1000000000400020C54400000545000007450000F1
:1000100000000000000000000000000000000000E0
:100020000000000000000000000000000945000082
:1000300000000000000000000B4500000D4500001E
:100040000F4500000F450000F94C00000F4500006F
:100050000F450000000000000F4500000F450000A4
:100060000F4500003D4700000F4500000F45000010
:100070000F4500000F4500000F4500000F45000030
:100080000F4500009D4D00000F4500000F4500008A
:100090000F4500000F4500000F4500000F45000010
:1000A0000F4500000F4500000000000000000000A8
:1000B0000000000000000000000000000000000040
:1000C000054B0648033310B51B1A062B03D9044B06
:1000D000002B00D0984710BDE4010020E40100206F
:1000E000000000000648074910B5091A8910CB0F17
:1000F0005918491003D0044B002B00D0984710BD6D
:10010000E4010020E40100200000000010B5074CCD
:100110002378002B09D1FFF7D3FF054B002B02D02A
:10012000044800E000BF0123237010BDE40100205B
:100130000000000070740000094B10B5002B03D0C4
:100140000849094800E000BF08480368002B02D1B5
:10015000FFF7C8FF10BD064B002BF9D09847F7E713
:1001600000000000E801002070740000E0010020A1
:1001700000000000164B002B00D1144B9D4640227E
:1001800092029A1A924600218B460F461348144A4F
:10019000121A05F072F80F4B002B00D098470E4B47
:1001A000002B00D098470020002104000D000D48CE
:1001B000002802D00C4800E000BF05F01BF820002A
:1001C000290004F0B1FD04F0EFFFC0460000080074
:1001D000004000200000000000000000E4010020BA
:1001E000E420002000000000000000000123034084
:1001F0000200181E04D1042A03D91068000900E087
:100200000020704710B50400FFF7F0FF0300002046
:1002100083420BD0013B9B00181DE2181279002A83
:1002200003D001338342F8D100E0180010BD012251
:10023000016810B5114201D0002903DA102000F046
:10024000E3F903E04910062001F004FF10BD016846
:1002500010B5CB0701D5002903DA102000F0D4F93E
:1002600006E04910033189100022052001F0F2FE5A
:1002700010BD70B50568AB0728D1042D26D90F2312
:100280002A6846681340062B09D12800FFF7AEFF05
:10029000012383421DDC9A00AE500133F9E7052BA0
:1002A00014D1F30703D4132000F0AEF912E0761056
:1002B000FF2EF8D82800FFF799FF2C1D230080009F
:1002C0002018984205D91E700133FAE70B2000F080
:1002D0009BF9002070BD70B50468E30701D41120BC
:1002E0002DE04568AB0729D1042D27D90F262B68AF
:1002F00064101E40062E0BD1002C04DD2800FFF7F1
:1003000075FF844201DD122019E0A400605918E055
:10031000331F012B12D82800FFF768FF8000042E3E
:1003200002D12800FFF76EFF002CECDDA042EADBD3
:1003300001232C19E0784000184302E00B2000F064
:1003400063F970BDF8B5012304681C4201D1112086
:100350002FE00325466835402AD1042E28D90F23E3
:100360003268641087681340062B0BD1002C04DD23
:100370003000FFF73BFF844201DD122019E0A400AA
:10038000A75113E0052B13D1002CF6DD3000FFF749
:100390002DFF80008442F0DC01231F4201D1132095
:1003A00007E07F10FF2FFAD83419E770280002E029
:1003B0000B2000F029F9F8BD006810B5830717D1AC
:1003C000042815D90F2302681340062B02D1FFF72A
:1003D0000DFF0BE0052B05D1FFF708FFC00001233F
:1003E000184308E0042B03D1FFF70CFF4000F6E7A9
:1003F0000B2000F009F910BD10B50324006804407B
:1004000006D1042804D90F2302681340042B01D01D
:100410000E2011E001F05AFE0378233B5942594166
:1004200010224018210005F001FC80239B05C21812
:10043000054B9A4203D9142000F0E6F802E00123AC
:100440004000184310BDC046FFFFFF3F10B5012418
:100450000368234202D04268224203D10D2000F0FB
:10046000D3F808E004495B1052101B070A401343FD
:1004700018684000204310BDFCFFFF0F01210368F6
:1004800010B50B4205D042680A4202D0806808428B
:1004900003D10D2000F0B8F808E005495B105210B8
:1004A0001B070A40401013431860002010BDC046CF
:1004B000FCFFFF0F012303400200181E01D0501063
:1004C00002E00D22014B1A707047C0460002002066
:1004D000012303400200181E04D1042A03D9106826
:1004E000000900E00020704770B50D000400FFF720
:1004F000EFFF86002800FFF7EBFF830000209E42FD
:100500000ED1231D9E1904351A009E4207D9297861
:100510001278013301358A42F6D0002000E0012034
:1005200070BD0000F0B585B00393019002912D4E8F
:100530002D4B002A02D002223270013A00251A60A7
:100540001B68F554019B9D424ADA029AAB00D058D1
:10055000254B1C68C8239B0037191C1B012318421C
:1005600002D04310214A1FE0214A002802D004286B
:1005700005D1204A2100380005F046FA18E0042889
:1005800010D90F2302681340042B04D101F09EFD03
:10059000194A030008E0062B05D1FFF799FF174A17
:1005A000030001E00123164A2100380005F02CFA6F
:1005B000300005F08FFA039B0B4A002B01D110602D
:1005C0000CE0019B013B9D42F9DA0E4B9842F6DCB0
:1005D000431C1360202232540022F2540135B1E74B
:1005E00005B0F0BD0C02002008020020F9690000EF
:1005F000CC690000D2690000006D0000D7690000DE
:10060000E86900001F030000014B187000207047CC
:100610000002002070B502F07BFE094C0100251D90
:100620001F22280005F05DFA280005F053FA042384
:1006300004308008000118432060200070BDC046CF
:100640002C050020C368F0B59D00836887B05D1954
:10065000030018330393036902909F00039BDF1983
:1006600043699E000093039B9E19D24B1B78002B7D
:100670000FD17F222B68D0491C1213409B005B587E
:1006800000960435019235E0CA4B1B78002B29D027
:10069000009E029BC74C9B6821780093EA1A029B3C
:1006A00092109B7812021A43029B587802F0BCFB0E
:1006B0000023029A2370137000960497029B039AFA
:1006C0009B68ED1A0193029BAD10DD60049B9F1A9D
:1006D000029BBF101F61009B9B1A029A9B105361E3
:1006E00001F005FC2B68019A1C121340B24A9B00D2
:1006F0009B5804359F46029B587802F08DFB0023DF
:10070000029A1370D9E7039B3A1DD11AA94B8B2982
:1007100003DD1A22009E1A70BBE71B783C60002B99
:1007200002D0009E1700B4E72B6801991C120B4001
:10073000A1499B005B5817000435DBE7039B3A1D7A
:10074000D11A9C4B8B2903DD1A22009E1A70A0E758
:1007500028681B78291D3860002B03D0009E1700E5
:100760000D0096E76B6801991C120B4092499B00A3
:100770005B5817000835BDE7039B3A1DD11A8D4B16
:100780008B2903DD1A22009E1A7082E7A4001B78D1
:100790002C193C60002B02D0009E170079E72B68D3
:1007A00001991C120B4084499B005B5817000435CB
:1007B000A0E7039B3A1DD11A7E4B8B2903DD1A2239
:1007C000009E1A7065E77D48A40021581B783960A7
:1007D000002B02D0009E17005BE72B6801991C12CA
:1007E0000B4075499B005B581700043582E7043FB6
:1007F000724B3A68A400E2506E4B1B78002B01D07C
:10080000009E46E72B68019A1C1213406A4A9B001F
:100810009B5804356EE7694BA600F058FFF74AFE77
:10082000043F04003868FFF745FE24180120634B9D
:1008300064000443F4505F4B1B78002B01D0009EF2
:1008400027E72B68019A1C1213405B4A9B009B58B8
:1008500004354FE7039B3A1DD11A564B8B2903DD14
:100860001A22009E1A7014E70098039C0121A042EE
:1008700002D901000C3909681B783960002B02D0BD
:10088000009E170005E72B6801991C120B404A498E
:100890009B005B58170004352CE7039B3A1DD11AC7
:1008A000444B8B2903DD1A22009E1A70F1E6009951
:1008B000039881420AD90B000C3B1B6840495B102E
:1008C0006418E41A009BA400E35802E01821197090
:1008D00000233B60374B1B78002B02D0009E170093
:1008E000D7E62B6801991C120B4033499B005B58DB
:1008F00017000435FEE6009B039A93420BD90C3B8C
:1009000019682F4B043FE3184910591A3A68009BA5
:100910008900CA5002E01822264B1A70254B1B781A
:10092000002B01D0009EB4E62B68019A1C121340E4
:10093000214A9B009B580435DCE6009B039A9342B6
:100940001CD9009E1E4B0C3EE4183368009A5B10C5
:10095000E31A9B009858FFF7ADFD043F04903868F8
:10096000FFF7A8FD3168049B4910611A012418188B
:100970004000009B89002043C85002E018220D4B24
:100980001A700C4B1B78002B01D0009E81E62B685F
:10099000019A1C121340084A9B009B580435A9E693
:1009A000039B3A1DD11A034B8B290BDD1A22009EA3
:1009B0001A706EE600020020CC6700004C1F002079
:1009C000FDFFFF3F0099A40061581B783960002BA0
:1009D00002D0009E17005CE62B6801991C120B40A8
:1009E000CF499B005B581700043583E6043F009B0A
:1009F0003A68A400E250CB4B1B78002B01D0009E3C
:100A000047E62B68019A1C121340C54A9B009B586D
:100A100004356FE6009BA4001C192368043F386866
:100A20005E10FFF747FD36180120BE4B76001B789D
:100A300006432660002B01D0009E2AE62B68019A0F
:100A40001C121340B64A9B009B58043552E6039B88
:100A5000A4003F1BB34CBB420DD82378002B01D020
:100A6000009E16E62B68019A1C121340AC4A9B00AC
:100A70009B5804353EE6AC4801F09EFA2378002BE3
:100A800001D0009E05E62B68019A1C121340A44A6F
:100A90009B009B5804352DE6A300ED18002C00DACE
:100AA0000BE6A04B1B78002B01D0009EF1E52B68D4
:100AB000019A1C1213409A4A9B009B58043519E670
:100AC0003B1F04931B680593042B04D1A300ED186E
:100AD000002C00DAF2E5934B1B78002B02D0009E2D
:100AE000049FD6E52B68019A1C1213408C4A9B0088
:100AF0009B58049F0435FDE53B1F04931B68059339
:100B0000002B04D1A300ED18002C00DAD6E5854BAC
:100B10001B78002B02D0009E049FBAE52B68019A37
:100B20001C1213407E4A9B009B58049F0435E1E54C
:100B30003A1F13685B10013B002B07DD01215B00AE
:100B4000A4000B4304972D191360B7E5754B1700EC
:100B50001B78002B01D0009E9BE52B68019A1C128C
:100B600013406F4A9B009B580435C3E53A00039B32
:100B70000C32D31A8B2B04DD1A226A4B009E1A709A
:100B800087E5FF2361005B000B4001210B433B60C5
:100B9000029B03989B6824120493ED1A029BAD10EC
:100BA0009B782D021D43009B8D401B1A9B108B4090
:100BB0000B43BB60029B0D437D609C70E4B25B4BBA
:100BC000E4000299E35816008B6056490978002921
:100BD00003D008331D0017005BE51D0001999B68D9
:100BE0000C351C120B404E499B005B5800921700BD
:100BF00080E53B1F1E68039A009B93422AD104970D
:100C00000A20F30716D4B3070DD1042E0BD90F23F6
:100C100032681340042B06D1300001F057FA04F07B
:100C200059FF063006E00720042E03D0002E01D025
:100C300080208000643001F09FFE002801D1043D37
:100C40003CE5029B3100587802F000F90023029A3B
:100C5000137033E5009B009A0C3B1B6802995B10F4
:100C60009B005B421F00D3180C3B1E601300083B27
:100C70001B68083FD7195A108A70D2B22B49D2008C
:100C80005B0055589B0A029A9B009560ED18009BEB
:100C9000043B1E68039B7610B6009E19214B1B78FF
:100CA000002B00D0F5E42B68019A1C1213401C4A5B
:100CB0009B009B58009604351CE53B1F1868FFF706
:100CC000F9FBA40006003F1B1E2833DC00280EDCC5
:100CD000144B1B78002B01D0009EDAE42B68019A9C
:100CE0001C1213400E4A9B009B58043502E502F08B
:100CF000F5FA033E361802F0F1FA0D4B801B9842CC
:100D0000F9D8084B1B78002B01D0009EC1E42B685A
:100D1000019A1C121340024A9B009B580435E9E4D7
:100D2000CC67000000020020FC690000541700207E
:100D30009F8601000123029A137002F0CFFA029BF2
:100D40000A3886195E60B8E43B1F1868FFF7B2FBEB
:100D5000A40004903F1B00280EDCCF4B1B78002B17
:100D600001D0009E95E42B68019A1C121340CB4AD7
:100D70009B009B580435BDE4C94B049A009E9A42DF
:100D800003DD1D22C44B1A7083E40123029A137001
:100D900002F0A4FAFA23049A9B005343029A0A3BF6
:100DA0001B18536089E4A300FF1A002320001A00D7
:100DB0003900FFF7B7FBBB4EBB4C3168200001F098
:100DC00091FF3168200002F048F8B34B1B78002BEC
:100DD00001D0009E5DE42B68019A1C121340AF4ABB
:100DE0009B009B58043585E4AB4BA4001B783F1B4C
:100DF000002B01D0009E4CE42B68019A1C1213407A
:100E0000A64A9B009B58043574E401F0FBFD01F0F9
:100E10006EF83B1F1868002823D1083B1868C307E9
:100E200001D5401016E083070FD104280DD90F23F8
:100E300002681340062B02D1FFF74AFB0AE0052B9C
:100E400003D1FFF745FB800004E01922924B009E7E
:100E50001A701EE43A0001214300083A0B43136064
:100E600001E040100138002832DD01224300134325
:100E7000391F0B603B00083B1B681341181A3B00ED
:100E80000C3B1B68134203D08018A400904015E06F
:100E9000990717D1042B15D90F211E683140062957
:100EA00006D101308000C358009AA400A35010E07E
:100EB000052907D118180079A4004000009B1043B1
:100EC000E05006E01922744B009E1A70FFF7E1FB18
:100ED0000435714B1B78002B02D0009EFFF7D9FB25
:100EE0002B68019A1C1213406C4A9B009B580435D6
:100EF000FFF700FCA300039AFB189B1A8B2B01DC65
:100F0000002205E01A22644B009E1A70FFF7C1FB15
:100F1000631E002C03DD3A601C000437F8E75E4BCB
:100F20001B78002B02D0009EFFF7B3FB2B68019AC1
:100F30001C121340594A9B009B580435FFF7DAFBFB
:100F4000A3009C46F81A002C04DC1C22524B0026FD
:100F50001A7015E0002103685B1001268A00825890
:100F6000164003D10D224C4B1A7009E052109342E7
:100F700000DD130001318C42EFDC01265B001E43D3
:100F80006346FF1A444B06601B780437002B02D0DF
:100F9000009EFFF77EFB2B68019A1C1213403F4A0C
:100FA0009B009B580435FFF7A5FBA3009C46F81A4D
:100FB000002C04DC1C22384B00261A7015E000219E
:100FC00003685B1001268A008258164003D10D2267
:100FD000314B1A7009E05210934200DA13000131CC
:100FE0008C42EFDC01265B001E436346FF1A2A4B4E
:100FF00006601B780437002B02D0009EFFF749FBE8
:101000002B68019A1C121340244A9B009B580435FC
:10101000FFF770FB3B00083B1868FFF74BFA3B1FDC
:1010200004901868FFF746FA049AA600BC1B002338
:10103000824200DA04332360174BBF1B1B7804374E
:10104000002B02D0009EFFF724FB2B68019A1C1294
:101050001340124A9B009B580435FFF74BFBA3003B
:10106000FE1A04933B00083B1868FFF723FA3B1F66
:1010700004001868FFF71EFAE20FC317A04253419D
:101080009B003360049BFF1A034B04371B78002B33
:101090000CD0009EFFF7FDFA00020020CC67000094
:1010A00080EE3600080200200C0200202B68019A16
:1010B0001C121340D84A9B009B580435FFF71AFBBB
:1010C0003B00083B18683B1F1968A300884202D107
:1010D000FB1A042222E004281ED90122104201D06A
:1010E000114219D10326304215D10F2302681A404C
:1010F000042A10D131420ED104290CD90A681340B8
:10110000042B08D1FFF7F0F9431E9841A600BE1B3F
:101110008000306003E0A3000022FB1A1A60BF4B7E
:10112000A4001B783F1B0437002B02D0009EFFF762
:10113000B0FA2B68019A1C121340B74A9B009B58C7
:101140000435FFF7D7FA3B00083B18683B1F1968C6
:10115000A300884202D1FB1A002223E004281FD9F1
:101160000122104201D011421AD10326304216D179
:101170000F2302681A40042A11D131420FD10429E9
:101180000DD90A681340042B09D1FFF7ADF903000C
:1011900058425841A600BE1B8000306003E0A30007
:1011A0000422FB1A1A609D4BA4001B783F1B0437D6
:1011B000002B02D0009EFFF76CFA2B68019A1C12DC
:1011C0001340954A9B009B580435FFF793FAA30000
:1011D000FE1A04933B00083B1868FFF76BF93B1FAE
:1011E00004001868FFF766F9E217C30F8442534101
:1011F0009B003360049BFF1A884B04371B78002B3D
:1012000002D0009EFFF745FA2B68019A1C1213408A
:10121000814A9B009B580435FFF76CFA3B00083B62
:101220001868FFF747F93B1F04901868FFF742F969
:10123000049AA600BC1B0023824200DD0433236015
:10124000764BBF1B1B780437002B02D0009EFFF7A4
:1012500020FA2B68019A1C1213406F4A9B009B587E
:101260000435FFF747FA3B1F1B686C4AA400042BA8
:1012700002D13B1B002103E0002B03D104213B1BC7
:10128000196001E00C23137013783F1B0437002B07
:1012900002D0009EFFF7FDF92B68019A1C12134043
:1012A0005D4A9B009B580435FFF724FAA300FC1A03
:1012B00004933B00083B1868FFF7FCF83B1F06004F
:1012C0001868FFF7F7F836180120049B7600FF1A1C
:1012D000524B06431B7826600437002B02D0009E39
:1012E000FFF7D7F92B68019A1C1213404A4A9B005A
:1012F0009B580435FFF7FEF9A300FE1A04933B0048
:10130000083B1868FFF7D6F83B1F04001868FFF782
:10131000D1F8241A0120049B6400FF1A3F4B0443B8
:101320001B7834600437002B02D0009EFFF7B1F920
:101330002B68019A1C121340374A9B009B580435B6
:10134000FFF7D8F9A300FC1A04933B00083B186888
:10135000FFF7B0F83B1F06001868FFF7ABF84643ED
:101360000120049B7600FF1A2C4B06431B78266055
:101370000437002B02D0009EFFF78BF92B68019AEF
:101380001C121340244A9B009B580435FFF7B2F906
:101390003B00083B1868FFF78DF83B1F0490186866
:1013A000FFF788F80100049803F0C6FD0123A400AC
:1013B0003E1B370040001843184B30601B78043741
:1013C000002B02D0009EFFF764F92B68019A1C12D3
:1013D0001340114A9B009B580435FFF78BF93B00E3
:1013E000083B1868FFF766F83B1F04901868FFF782
:1013F00061F80100049803F085FE0123A4003E1B60
:10140000370049001943054B31601B780437002B26
:1014100006D0009EFFF73DF9CC67000000020020D7
:101420002B68019A1C121340E74A9B009B58043515
:10143000FFF760F93B1F1868FFF73CF8C317C018A7
:101440005840012340001843E04BA4001B783E1B8A
:101450003060371D002B02D0009EFFF71AF92B6871
:10146000019A1C121340D84A9B009B580435FFF781
:1014700041F9A300FE1A05933068012C03D1FFF750
:1014800019F8049008E0FFF715F804007068FFF7FA
:1014900011F80130031B0493049B002B01DC012392
:1014A000049304F063FA049903F02CFE0C19012153
:1014B000059B6400FF1AC54B0C431B78346004374E
:1014C000002B02D0009EFFF7E4F82B68019A1C1253
:1014D0001340BD4A9B009B580435FFF70BF9A4004D
:1014E0003E1B3000FEF788FFB84B30601B78371D7D
:1014F000002B02D0009EFFF7CCF82B68019A1C123B
:101500001340B14A9B009B580435FFF7F3F8A30042
:10151000FE1A04933B00083B1868FEF7CBFF3B1F05
:1015200004001868FEF7C6FF04400120049B640015
:10153000FF1AA64B04431B7834600437002B02D0FB
:10154000009EFFF7A6F82B68019A1C1213409E4AD2
:101550009B009B580435FFF7CDF8A300FC1A0493B9
:101560003B00083B1868FEF7A5FF3B1F0600186804
:10157000FEF7A0FF06430120049B7600FF1A934B61
:1015800006431B7826600437002B02D0009EFFF72D
:1015900080F82B68019A1C1213408B4A9B009B58C1
:1015A0000435FFF7A7F8A300FC1A04933B00083B9F
:1015B0001868FEF77FFF3B1F06001868FEF77AFFEA
:1015C00046400120049B7600FF1A804B06431B789F
:1015D00026600437002B02D0009EFFF75AF82B68D4
:1015E000019A1C121340784A9B009B580435FFF760
:1015F00081F83B1F1868FEF75DFFC04301234000E0
:101600001843724BA4001B783E1B3060371D002B23
:1016100002D0009EFFF73DF82B68019A1C12134080
:10162000694A9B009B580435FFF764F8A300FE1A33
:1016300004933B00083B1868FEF73CFF3B1F040087
:101640001868FEF737FF8440012364001C43049BA5
:101650003460FF1A5D4B04371B78002B02D0009ECC
:10166000FFF717F82B68019A1C121340564A9B008B
:101670009B580435FFF73EF8A300FE1A04933B0085
:10168000083B1868FEF716FF3B1F04001868FEF7BA
:1016900011FF0441012364001C43049B3460FF1AC2
:1016A0004A4B04371B78002B02D0009EFEF7F1FF57
:1016B0002B68019A1C121340434A9B009B58043527
:1016C000FFF718F8A4003E1B3000FEF7B0FD3F4BBB
:1016D00030601B78371D002B02D0009EFEF7D9FF2B
:1016E0002B68019A1C121340374A9B009B58043503
:1016F000FFF700F8A4003E1B3000FEF7A8FD334BB7
:1017000030601B78371D002B02D0009EFEF7C1FF12
:101710002B68019A1C1213402B4A9B009B580435DE
:10172000FEF7E8FFA4003F1B3800FEF7A2FD274BA1
:101730001B78002B02D0009EFEF7ABFF2B68019AAE
:101740001C121340204A9B009B580435FEF7D2FF21
:10175000A4003E1B3000FEF7BEFD1C4B30601B7822
:10176000371D002B02D0009EFEF793FF2B68019AD5
:101770001C121340144A9B009B580435FEF7BAFF15
:10178000A4003F1B3800FEF7DDFD104B1B78002B3B
:1017900002D0009EFEF77DFF2B68019A1C121340B9
:1017A000094A9B009B580435FEF7A4FFA4003E1B8A
:1017B0003000FEF701FE054B30601B78371D002B13
:1017C00006D0009EFEF765FFCC67000000020020F7
:1017D0002B68019A1C121340E64A9B009B58043563
:1017E000FEF788FF039A3B1D0493E34C9B1A8B2B57
:1017F00004DD1A23009E2370FEF74BFF01F078FDF5
:1018000001234000184323783860002B03D0009E4A
:10181000049FFEF73EFF2B68019A1C121340D54A25
:101820009B009B58049F0435FEF764FF039A3B1D01
:101830000493D14C9B1A8B2B04DD1A23009E23703A
:10184000FEF727FF01F04AFDCC4B40001840012372
:10185000184323783860002B03D0009E049FFEF7C6
:1018600018FF2B68019A1C121340C24A9B009B5818
:10187000049F0435FEF73EFFA4003E1B3000FEF738
:10188000E5FDBD4B30601B78371D002B02D0009E5C
:10189000FEF7FFFE2B68019A1C121340B54A9B000D
:1018A0009B580435FEF726FFA4003F1B3800FEF7C7
:1018B000E5FDB14B1B78002B02D0009EFEF7E9FE40
:1018C0002B68019A1C121340AA4A9B009B580435AE
:1018D000FEF710FFA300FB1A0493012320001A0057
:1018E0000499FEF71FFEA64C2068643001F044F80E
:1018F000002816D0029B21685A78A24801F0BBFA52
:1019000015E0A300FB1A0493200001230022049990
:10191000FEF708FE9A4C2068643001F02DF800288C
:1019200002D1043DFEF7C9FE964801F03FF90123BC
:10193000029A137001F0D2FC9622236852000633FB
:1019400053431818029B5860FEF7B8FEFEF762FE7C
:10195000894BA4001B783E1B3060371D002B02D042
:10196000009EFEF796FE2B68019A1C121340814AD6
:101970009B009B580435FEF7BDFEA4003E1B3000C3
:1019800001F0EAFC7C4B30601B78371D002B02D045
:10199000009EFEF77EFE2B68019A1C121340754ACA
:1019A0009B009B580435FEF7A5FEA4003E1B3000AB
:1019B00001F0D4FC704B30601B78371D002B02D037
:1019C000009EFEF766FE2B68019A1C121340694ABE
:1019D0009B009B580435FEF78DFEA4003E1B300093
:1019E00001F0BEFC644B30601B78371D002B02D029
:1019F000009EFEF74EFE2B68019A1C1213405D4AB2
:101A00009B009B580435FEF775FEA4003F1B380071
:101A100001F0C4FC584B1B78002B02D0009EFEF74F
:101A200038FE2B68019A1C121340524A9B009B58A7
:101A30000435FEF75FFEA4003E1B300001F0D0FC31
:101A40004D4B30601B78371D002B02D0009EFEF7F7
:101A500020FE2B68019A1C121340464A9B009B589B
:101A60000435FEF747FEA4003F1B380001F0EAFCF6
:101A7000414B1B78002B02D0009EFEF70AFE2B681C
:101A8000019A1C1213403B4A9B009B580435FEF7F9
:101A900031FE0121200001F0BDFC374B1B78002BEB
:101AA00002D0009EFEF7F5FD2B68019A1C12134030
:101AB000304A9B009B580435FEF71CFE0021200095
:101AC00001F0A8FC2C4B1B78002B02D0009EFEF7E7
:101AD000E0FD2B68019A1C121340264A9B009B587C
:101AE0000435FEF707FEA4003E1B300001F0C8FCE1
:101AF000214B30601B78371D002B02D0009EFEF773
:101B0000C8FD2B68019A1C1213401A4A9B009B586F
:101B10000435FEF7EFFDA4003E1B300001F0C4FCCD
:101B2000154B30601B78371D002B02D0009EFEF74E
:101B3000B0FD2B68019A1C1213400E4A9B009B5863
:101B40000435FEF7D7FDA4003F1B380001F086FCEA
:101B5000094B1B78002B02D0009EFEF79AFD2B68E4
:101B6000019A1C121340034A9B009B580435FEF750
:101B7000C1FDC046CC67000000020020FEFFFF7FD1
:101B8000080200200C020020A4003F1B380002F0D5
:101B900071F9D84B1B78002B02D0009EFEF779FD1F
:101BA0002B68019A1C121340D34A9B009B580435A2
:101BB000FEF7A0FDA4003E1B300002F0CBF9CD4B98
:101BC00030601B78371D002B02D0009EFEF761FDB0
:101BD0002B68019A1C121340C74A9B009B5804357E
:101BE000FEF788FDA4003F1B380002F013F9C14B3B
:101BF0001B78002B02D0009EFEF74BFD2B68019A4C
:101C00001C121340BC4A9B009B580435FEF772FD22
:101C1000A4003E1B300002F013F9B64B30601B7875
:101C2000371D002B02D0009EFEF733FD2B68019A72
:101C30001C121340B04A9B009B580435FEF75AFD16
:101C4000A4003F1B380001F01FFFAA4B1B78002B9C
:101C500002D0009EFEF71DFD2B68019A1C12134056
:101C6000A54A9B009B580435FEF744FDA4003F1B8A
:101C7000380001F01FFF9F4B1B78002B02D0009E05
:101C8000FEF707FD2B68019A1C1213409A4A9B002D
:101C90009B580435FEF72EFDA4003F1B380001F0D1
:101CA00019FF944B1B78002B02D0009EFEF7F1FC2D
:101CB0002B68019A1C1213408F4A9B009B580435D5
:101CC000FEF718FDA4003F1B380001F02BFF894BE5
:101CD0001B78002B02D0009EFEF7DBFC2B68019ADC
:101CE0001C121340844A9B009B580435FEF702FDEA
:101CF000A300FE1A31002000049302F06CF9049B4B
:101D00003060FF1A7B4B04371B78002B02D0009EFB
:101D1000FEF7BFFC2B68019A1C121340764A9B0009
:101D20009B580435FEF7E6FCA300FE1A31002000A4
:101D3000049302F068F9049B3060FF1A6D4B04377E
:101D40001B78002B02D0009EFEF7A3FC2B68019AA3
:101D50001C121340684A9B009B580435FEF7CAFCCE
:101D6000A300FE1A31002000049302F00EF9049B38
:101D70003060FF1A5F4B04371B78002B02D0009EA7
:101D8000FEF787FC2B68019A1C1213405A4A9B00ED
:101D90009B580435FEF7AEFCA300FE1A310020006C
:101DA000049302F00BF9049B3060FF1A514B043787
:101DB0001B78002B02D0009EFEF76BFC2B68019A6B
:101DC0001C1213404C4A9B009B580435FEF792FCB2
:101DD000A4003F1B380001F0CDFE464B1B78002BC2
:101DE00002D0009EFEF755FC2B68019A1C1213408E
:101DF000414A9B009B580435FEF77CFCA300FF1A68
:101E00003900200001F06CFF3A4B1B78002B02D008
:101E1000009EFEF73EFC2B68019A1C121340364AC6
:101E20009B009B580435FEF765FCA4003E1B300068
:101E300001F022FF2F4B30601B78371D002B02D0A2
:101E4000009EFEF726FC2B68019A1C1213402A4ABA
:101E50009B009B580435FEF74DFCA300FF1A390088
:101E6000200001F0E7FE234B1B78002B02D0009EE0
:101E7000FEF70FFC2B68019A1C1213401E4A9B00B0
:101E80009B580435FEF736FCA300FF1A39002000EA
:101E900000F0F6FC174B1B78002B02D0009EFEF7DB
:101EA000F8FB2B68019A1C121340134A9B009B58A5
:101EB0000435FEF71FFCA300FE1A31002000049336
:101EC00000F0DEFC049B3060FF1A0A4B04371B78DD
:101ED000002B02D0009EFEF7DCFB2B68019A1C123F
:101EE0001340054A9B009B580435FEF703FC07B0DE
:101EF000F0BDC04600020020CC6700000023F7B50B
:101F00005A1E0192002B07DA01F06AFC00F024FF50
:101F100000F0D6FF6423019300263000194B1968A6
:101F20008E4201DB019BEBE7174B1A6801329142AD
:101F300000DC0022A0241A601D68144F6C43E35D8E
:101F4000002B1DD0E419022B16D0012B0ED1002836
:101F500001D101F0C3F9A0226A430C4B0C499B1834
:101F60005B68C31A8B4201D80223BB54A0235D4394
:101F7000064BEB5C022B03D12000FEF763FBD1E79D
:101F80000136CBE7040200200000002014110020DD
:101F90009F860100054B01211A68054B1A6000233A
:101FA000044AD1500433642BFBD1704758050020FC
:101FB000500500204C1F002000B59BB002000549D1
:101FC00001A803F053FD01A800F00CFE00F078FF1B
:101FD000FCE7C0460C6A000037B5174D04002868BE
:101FE000002801D003F036F9A400200003F028F9FE
:101FF0002860002801D1114809E001AB984208D2BD
:102000000F4B02196B440193934202D20D48FFF724
:10201000D3FF042802D808302860083C2B680A4AFD
:102020001C191360094B01211C600023084AD15080
:102030000433642BFBD137BD580500201D6A000016
:102040001CFCFFFF4D6A00005005002054050020D5
:102050004C1F002070B50D4D0D4E2B684C1CA4007C
:1020600036681C19B44203D90A20FEF7CDFA0BE0FA
:102070002C601D00AC4201D904C5FBE70F22090109
:10208000104008431860180070BDC046500500207D
:10209000540500200322CB1C70B50C00D917114049
:1020A000C9180500891000220420FFF7D3FF002380
:1020B000A34204DAE95CC21811710133F8E7E14385
:1020C0000023C917214041180B7170BD10B583075B
:1020D00006D1042804D90F2304C81340042B03D0CD
:1020E0000E20FEF791FA014810BDC046546B000067
:1020F00030B502248025094B094AED009C505C59FB
:10210000002CFCD0A124E400884204D28025ED00FC
:1021100018514019F8E70021995030BD00E0014006
:102120000405000010B5002804D19020922100027F
:10213000890203E0922080218002C902FFF7D8FFC4
:1021400010BD002802D092239B0201E090231B02C5
:102150001B6800201A0E532A01D11B02180A70476F
:1021600030B501248025064A064BED00D450545961
:10217000002CFCD001600021014AD15030BDC04686
:1021800000E001400405000010B5002802D09220B4
:10219000800201E090200002A6230902DB05090A63
:1021A0001943FFF7DDFF10BDF0B5012480250300C2
:1021B0000F4F08000F49ED007C507C59002CFCD0DB
:1021C0009C46002810DD5478167893782402344316
:1021D0001B0423431C00D37801381B0623436446A9
:1021E00008C40432A446ECE700237B50F0BDC0468F
:1021F00000E001400405000070B505004B680A00CE
:102200009C1C2100FFF7D0FFA000281870BD000023
:10221000154B1B68002B04D080219223C9029B021E
:1022200003E09221902389021B02002807D1191D87
:102230005B6802001B0E522B14D10A0012E0002230
:1022400081420FD903681B0E522B0BD14368023316
:102250009B00C318994205D91A68110E0022522911
:1022600000D11A00100070475C0700208022F0B5F2
:10227000520085B00021624802F0FFFF8022002159
:102280005200604802F0F9FF5F4B1B681A0002938E
:1022900053425A4110000392FFF744FF029B002B68
:1022A00001D15A4C00E05A4C0020FFF7B1FFFF2744
:1022B0000500002D00D194E02B681A121B143A403F
:1022C0003B4001921A000A3A092A43D84C4B019A22
:1022D000995C002900D07FE010224E4802F0CDFF2B
:1022E0002E00336801991A123A40914217D11A14FC
:1022F0003A400B2A06D0132A0CD00A2A0FD1454B9C
:102300001E600CE03B40022B09DC424A9B00D318C4
:102310005E6004E0102200213E4802F0AEFF300073
:10232000FFF776FF061EDCD13A4B196800290FD063
:102330002000FFF761FF0400374E3168002903D009
:102340002000FFF759FF0400344B0436B342F4D1A8
:102350002B4B3EE0143B092B3ED82A4B019A995C4B
:10236000002939D108222E4802F087FF2E00336859
:102370001A143A40152A0BD01D2A11D0142A14D150
:10238000019A1B123B409A420FD1254B1E600CE074
:10239000019A1B123B409A4207D1214B5E6004E038
:1023A000082200211E4802F068FF3000FFF730FFCE
:1023B000061EDCD11A4E3168002909D02000FFF733
:1023C0001BFF71680400002902D0FFF715FF04000D
:1023D0000C4B0121019A99542800FFF719FF0500C1
:1023E00067E70298FFF7ADFE411C0398FFF7CCFEAC
:1023F000054B039A1A600B4B1C6005B0F0BDC0463C
:102400005C0600205C0500205C07002004480200F8
:1024100004900000B01F0020B41F0020C01F002047
:10242000C01F00206007002070B50020FFF789FE64
:1024300004000120FFF785FE844200DA04000A4B05
:102440001E687542754128001D60FFF76BFE002E67
:1024500001D0064B00E0064B064A2800611C1360C1
:10246000FFF792FE70BDC0465C070020049000009C
:102470000448020060070020F8B50020FFF761FE65
:1024800007000120FFF75DFE3E00224D0643224C6F
:102490000CD180219020C9020002FFF729FE012102
:1024A0003000FFF771FE2E601C4B2FE0874208DDE5
:1024B000002392212B60194B89022360236800209E
:1024C00011E0012380212B60154BC9022360F5E741
:1024D0001A68551C18D0120E522A07D101205A68CA
:1024E000023292009B188B42F2D311E0002800D0F8
:1024F00023600C4C0C49200003F0E4FA200000F0AB
:10250000FFFEFFF791FF04E0002802D0236000E007
:102510002160F8BD5C0700206007002004900000E7
:102520000448020004200020C56A0000F0B585B010
:10253000039203220333DC1714402A4EE3189C1045
:10254000336801900291002B02D08022D20201E078
:1025500092229202244FA51C3B68AD005B199A425F
:1025600017D2FFF783FE3368002B02D08022D202FD
:1025700001E0922292023B685B199A4209D21B4CFD
:102580001B49200003F09EFA200000F0B9FE002055
:1025900026E0029B3E681B06190C6B461A7BA4239F
:1025A000DB051343019A0B431104FF22120411406F
:1025B00019433000FFF7D4FD3300301D08332100EC
:1025C00001933B60FFF7CCFD002C04D00A9A210058
:1025D0000198FFF7E9FD3000019B083D5D193D6062
:1025E00005B0F0BD5C07002060070020042000203B
:1025F000EE6A000070B59AB0FFF73EFFFF221F4C55
:10260000D2000021200002F038FE0020FFF700FE7B
:10261000FF25002600281AD003681A142A400A2A27
:1026200008D11A122A40FF2A0ED0D200A1180B712D
:10263000A05009E0132A07D11B122B40FF2B03D017
:10264000DB00E2181671E650FFF7E2FDE2E7FF213A
:102650000200C900235808305D1EAB41D2188842E1
:10266000F8D1074901A803F001FA01A800F0BAFA6D
:10267000044800F0B7FA1AB070BDC04654170020E5
:10268000156B00002D6B0000002070470120704783
:1026900000487047EC1F00200048704733F8FFFFE8
:1026A00010B50449044803F00DFA242303480360DD
:1026B00010BDC046E86B0000CC1F0020C81F0020E2
:1026C00000207047002070470020704700207047AE
:1026D000002070470020704700207047002070479E
:1026E0000020704710B5034A0E21034800F0B4F8EB
:1026F00010BDC04604000020ED6B0000044A0549EF
:102700001368C85401339B059B0D13607047C04686
:10271000680B002064070020114A70B51368114C43
:10272000984211DA015D451CFA39012906D8AB42FD
:1027300006DD2118497801391F2901D92800EFE762
:102740000100251A461C02D10023136006E0665CD6
:102750006E5401318B42FADC181A106070BDC0460D
:102760006C0B0020740B002010B500F0B7FD064B79
:102770001A68904201D200221A601B68C01A034BEB
:1027800083428041404210BD700B0020204E00006B
:1027900010B5094C094A2368126893420BD0084AC5
:1027A000D05C00F0D7FE002805D0236801339B05DC
:1027B0009B0D2360EDE710BD740F0020680B002017
:1027C0006407002010B50400064B074A1B68126816
:1027D0009B1ADB439B059B0DA34202DAFFF7D8FF50
:1027E000F2E710BD680B0020740F0020F7B506005B
:1027F0000191151E2FD05768B800441C0630FFF712
:10280000E1FFFB20FFF77AFF1C20FFF777FFF0B214
:10281000FFF774FFE0B22412FFF770FFE0B2FFF79A
:102820006DFF6B461879FFF769FF0026BE4212DA8A
:10283000B300EB189C680136E0B2FFF75FFF20128F
:10284000C0B2FFF75BFF2014C0B2FFF757FF200EA6
:10285000FFF754FFEAE7F7BD70B5074D2C68092C68
:1028600008DC0C236343054E01349851F31859607A
:102870009A602C6070BDC046780F00206820002050
:10288000F0B589B004900E0001284BDD284B086894
:102890000293830709D1042807D90F230268134044
:1028A000042B02D1FFF712FC0290214B70680393B6
:1028B000830709D1042807D90F2302681340042B8A
:1028C00002D1FFF703FC039000271A4B1A4D1B6837
:1028D0000593059B9F4225DA2B1F0299186803F088
:1028E000E7F800281BD12B686C6806930190019BC8
:1028F000069A934213DA20680399079403F0D8F8F4
:102900000834002807D131000498079B08315B6820
:102910000238984709E0019B01330193E7E701374B
:102920000C35D6E71B20FDF76FFE09B0F0BDC046A1
:10293000546B0000780F00206C20002010B501F0CF
:1029400043FA00F0C7FD00F033FEFFF7CBFE01F0C5
:1029500085FA01F077FB10BDC82210B5D200002126
:10296000034802F08AFC0022024B1A6010BDC046E8
:102970001411002004020020064B074A1B6812684D
:102980009B1ADB439B059B0D0122834200DC002246
:1029900010007047680B0020740F0020F8B5050088
:1029A0000C0016001F1E0ED10320FFF7E5FF0028C4
:1029B00027D0FA20FFF7A2FEE8B2FFF79FFEE0B2B1
:1029C000FFF79CFE1DE0501DFFF7D6FF002818D032
:1029D000FB20FFF793FEE8B2FFF790FEE0B2FFF7AF
:1029E0008DFEF0B2FFF78AFE3012C0B2FFF786FE0E
:1029F0003C00E31B9E4204DD2078FFF77FFE01349C
:102A0000F7E7F8BD70B50024A0250B4B1B689C426E
:102A10000EDA2A006243094BD3181A78002A05D02F
:102A20005978002311201A00FFF7B8FF0134ECE7B2
:102A3000FFF792FF70BDC046040200201411002071
:102A40000123F3B50400FFB00D0010001A420DD0B1
:102A500002AA1370431002A9537042121B0E4014B5
:102A60008A700B71C8700B00052273E003231340BA
:102A70001ED1042A1CD90F2201680A40042A17D14A
:102A8000023302AA1370FFF721FB060003F022F8BD
:102A9000F823FF33984200DD18000023834205DA53
:102AA00001335A1EB25C02A9CA54F7E7421C50E037
:102AB000042801D0002809D1032302AA0438137086
:102AC0004342434153701300022243E0002B45D19F
:102AD000042843D90F2102681140052912D104337B
:102AE00002A90B70F8231209FF3392009A4200DD0D
:102AF0001A00002393422BDA0133C118C97802AEC1
:102B0000F154F7E7062929D101390E00120956437D
:102B10000196F826019FFF36B7421FDC02AE3170E6
:102B20000136934213DA01270133990041583942A3
:102B300001D0394100E00A49012737700F12717046
:102B4000B7700F14090EF77031710536E9E7019A75
:102B5000013202AB29002000FFF720FF7FB0F3BD58
:102B600019FCFFFF70B5A023050000240D4A1800D2
:102B7000604380184178A94203D001340A2CF6D171
:102B80000FE0A022002102F078FB074A1368013B06
:102B9000A34200D11460002329001A001120FFF77E
:102BA000FDFE70BD141100200402002010B5B2B06B
:102BB00002236A460400137002F08CFFC72800DD70
:102BC000C7200023834205DA694601335A1EA25CFE
:102BD000CA54F7E7421C6B46FE211420FFF7DEFEC5
:102BE00032B010BD10B5B2B002236A4604001370B3
:102BF00002F070FFC72800DDC7200023834205DAFA
:102C0000694601335A1EA25CCA54F7E7421C6B4660
:102C1000FF211420FFF7C2FE32B010BDF7B5234BE1
:102C200006001B68A020009300232149009A9342CC
:102C30000ADA02005A438A185478B44202D1127850
:102C4000002A31D10133F1E70024A0231A006243A6
:102C500001920199164A55182F78002F06D0013499
:102C60000A2CF3D11348FFF7BDFF1DE0A022390065
:102C7000280002F002FB02230D4A0199EB60535435
:102C80000D4AF1008A58009B6E70AE70AA602F61E9
:102C90006F61A34202DC054B01341C60002331004C
:102CA0001A001020FFF77AFEF7BDC046040200208C
:102CB00014110020A86C00005417002010B5FFF775
:102CC000A1FE0024064BE200D3181B79043B012B24
:102CD00002D8E0B2FFF7A2FF0134FF2CF2D110BD01
:102CE00054170020F7B50E0000247F250190194BE2
:102CF000E200D1180979062901D0032926D1985874
:102D000083682B401C2B21D1C3681A002A40042A57
:102D10001CD102692A40192A18D11B0A01339B00D1
:102D20000C30C018FFF7D2F9070002F0D3FE0023E1
:102D3000B0420BD19E4206DD019AF95CD25C914211
:102D400004D10133F6E7E0B2FFF768FF0134FF2C4E
:102D5000CDD1F7BD5417002070B500F0BFFA184B65
:102D60001A68904201D200221A601A681549821A24
:102D70008A4223D91860002000F082FB444244417B
:102D8000604207240443002000F08EFB002810D08E
:102D9000082600250C4BEA00D3181B799C4201D071
:102DA000B34202D1E8B2FFF739FF0135FF2DF1D16F
:102DB00004E0631C02D001267642EAE770BDC046FB
:102DC000640B00200F2700005417002037B50024A3
:102DD0000500FFF717FE01A8019400F03FFB20005B
:102DE00000F068FE00F0FCFC00F072FB00F071FBEC
:102DF00000F038FF00F09EFA0548FFF7F3FEA54209
:102E000004D0FFF7C7F80348FFF7ECFE37BDC04614
:102E1000BD6C0000D56C0000002310B501001A0045
:102E20001120FFF7BBFD10BD07B56B461970694651
:102E30005A7013128B701314120ECB700A716B46FA
:102E4000010005221320FFF7A9FD07BD10B50A00F8
:102E500001001220FFF7F4FD10BD70B50500080059
:102E60000C003230FFF7AEFC2B00220000211B20AB
:102E7000FFF794FD70BD10B50C0003001100142085
:102E80002200FFF78BFD10BD70B506000020FFF794
:102E9000BFF90024FF25002810D003681A142A4027
:102EA000152A05D11B122B40B34204D1040002E0C5
:102EB0001D2A00D10024FFF7ABF9ECE7200070BD1C
:102EC000F0B580279DB0FFF763FCB94DB94C286879
:102ED000FF00391A201800F023FB2B680600C318E6
:102EE0002B60002B00D1DBE1002E0DDD2868391AA4
:102EF000201800F015FB2B6806001B182B6000F053
:102F0000EDF9AD4B1860EFE72378FA2B00D00CE118
:102F10002B68022B06DCFFF727FC002800D1BFE15D
:102F20000120B8E16078A5780238182800D9FAE0C5
:102F300001F06EFF0D1E22262932F93D676F75895B
:102F4000DAEFF9F9F9F9F9F9F9F9F9F9F300FF2DDF
:102F500000D1E8E02800FFF705FE00229749EB00CA
:102F60005A50CB181A7129000092130013204DE01B
:102F70002800FFF753FED6E02800FFF7F3FDD2E06C
:102F8000FFF79CFECFE0FFF73DFD0020FFF71EFF9F
:102F90008B48FFF727FEC6E0182D00D9C3E0894B08
:102FA000AA00D25829001520FFF74AFDBBE00024F3
:102FB0002000FFF769FF071E03D10134192CF7D158
:102FC000B1E0083002F086FD06000530FFF7FAFB9D
:102FD000FB20FFF793FB1D20FFF790FBE0B2FFF70C
:102FE0008DFBF0B2FFF78AFB3012C0B2FFF786FB11
:102FF0000025AE42E1DD7B19187AFFF77FFB013532
:10300000F7E700211D200B000A000091FFF78EFA60
:1030100089E000222900009213002720F6E700F043
:1030200077F903AC684A64210090684B200002F0F5
:10303000EBFC02232000237002F04CFD2300020071
:10304000002116206DE000245C4AE300D558002DD5
:1030500046D06B689E00701DFFF7B4FB2B00002567
:103060003200083321000120FFF798FC0020FFF711
:10307000CFF82E002F0000281DD0FF2103681A1260
:103080000A40A24214D11A140A400B2A07D10B405D
:103090000DD0012B09D0022B00D1FFE008E0132A4C
:1030A00006D100252E002F0002E0060000E00700F8
:1030B000FFF7AEF8DFE7002E04D032000121200038
:1030C000FFF794FB002D04D02A0002212000FFF717
:1030D0008DFB002F04D03A0000212000FFF786FB73
:1030E0000134FF2CB0D11EE0FFF78CFC002500243A
:1030F000290000942300220013200135FFF716FA5F
:10310000FF2DF4D1FF222100D2002C4802F0B5F8A7
:1031100009E00120FFF75AFE05E0002329001A000C
:103120001A20FFF73BFC0320B5E0FB2B00D0F7E6AD
:103130002A68042A00DCEEE62679E078244B360281
:1031400006439E4200DDEBE6331D9A4200DCE2E6D8
:10315000E35CFE2B00D0E3E66078A578731E1C28A4
:1031600068D007D8082835D01B285ED0012800D0A9
:1031700090E007E01E2800D17EE066D31F2800D132
:1031800080E087E0FF2D00D184E02800FFF7EAFC13
:1031900067790634B31E290000943A000A20FFF72D
:1031A000C5F9064BED00E8505D192F7172E0C0467D
:1031B0006C0B0020740B0020700B002054170020B3
:1031C000E56C00004C1F0020FC6C0000F76C000058
:1031D000F6030000182D5DD86079022813D003286B
:1031E0001BD0012856D1A71D7A78A479BB7812028A
:1031F00022431B0413431A00FB78AD001B06134344
:103200005B0003430EE0002B44DDB11EA01DFEF762
:1032100041FF244BAD00E8503CE0A379AD005A1EBD
:1032200093419B001F4AAB5034E0601D1900FFF72B
:1032300059FD2FE0FF2D2DD06279022A2AD80634BD
:10324000B31E009429000B2022E0632B00DD6323D2
:10325000002203A8934204DDA11849798154013268
:10326000F7E7D9430022C917194041180A70013302
:103270000090290015200BE005340094002229005D
:103280001E2005E0042B05D10022290005340094FE
:10329000FFF74CF9701DFFF73FFA01E0050007E763
:1032A0001DB0F0BD4C1F002000207047002070476B
:1032B000002070470020704701220020054B06497E
:1032C0001A61585003300431585080180831585052
:1032D0001A60704700800040040500000122034B83
:1032E0001A64A822D20098587047C0460080004057
:1032F00010B5FFF7F3FFFA21890001F093FD10BD2F
:1033000010B50100014801F037FB10BDA0100020EE
:10331000004870470C6D000070B5054E0400335C2A
:103320000D008B4202D001F04FFA355570BDC046FA
:103330007C0F002070B50024064D635D012B05D184
:103340000021200001F040FA0023635501341A2CBB
:10335000F2D170BD7C0F00200D20704735207047E2
:10336000036870B55B100120052B12D8094A9B0039
:103370009C58094D2B5D002B05D00021200001F049
:1033800023FA00232B55200001F0C8F80123400048
:10339000184370BD386D00007C0F002070B50368C5
:1033A00045685C106D1004D40B4B9D4202DD1D007E
:1033B00000E00025192C0DD8084E335D012B05D0F7
:1033C0000121200001F000FA0123335529002000DB
:1033D00001F032F970BDC046FF0300007C0F0020F1
:1033E00070B504686410192C0FD8094D2B5D002BA3
:1033F00005D00021200001F0E7F900232B55200023
:1034000001F016FA0423012800D00023180070BD33
:103410007C0F002070B504000D0019280ED8084E4E
:10342000335C012B04D0012101F0CEF90123335587
:10343000290020004D1EA94101F0E4F970BDC046ED
:103440007C0F0020436810B5191F4A424A410068AA
:1034500011004010FFF7DEFF10BD000037B56946D0
:103460000200064B684630CB30C11368042B02D1F2
:1034700000F030FB01E000F055FB37BD046D0000AB
:1034800010B5084C237D002B05D00021142001F03D
:103490009BF900232375142001F0CAF943425841D7
:1034A000800010BD7C0F002010B5084CA37D002BC0
:1034B00005D00021162001F087F90023A3751620FE
:1034C00001F0B6F943425841800010BD7C0F002046
:1034D0007047704710B5034A04210348FFF7BCF951
:1034E00010BDC04674000020FD6B0000E12110B546
:1034F0004902094801F087FAFFF7DEFE0A2001F0D1
:1035000007F80023FF21054A995401331A2BFBD1F8
:1035100000F0A8FB10BDC046A01000207C0F0020CA
:10352000F8B50B4E070030000D0001F0ABFA041E99
:10353000AC4200DD2C003D00EB1B9C4205DD300061
:1035400001F0AAFA28700135F6E72000F8BDC04660
:10355000A010002010B50100014801F05BFA10BD79
:10356000A01000200020704710B51E20FDF74CF879
:1035700010BD10B51E20FDF747F810BD10B51E2078
:10358000FDF742F8002010BD10B51E20FDF73CF8F5
:1035900010BD10B51E20FDF737F810BD10B51E2068
:1035A000FDF732F810BD10B51E20FDF72DF810BD47
:1035B00010B5034A08210348FFF74EF910BDC04675
:1035C00094000020506D00000123034A1360034A59
:1035D0001068984018437047A00F0020A80F0020E3
:1035E0001E2800D91A20084B8000C258012393409E
:1035F000064A07491360074A1160074A07491160E4
:10360000074A13607047C046EC7100009C0F002011
:1036100008050050B80F0020B00F00200C05005026
:1036200018050050F0B5EFF310810123194083F322
:103630001088134E134AB4461268013A9340124A56
:103640001468124A1568124A002B15D016680342F6
:103650000BD02660C046C046C046C046C046C046E5
:10366000C046C04616682E6004E067463E60166895
:10367000084F3E605B08E7E781F31088F0BDC04665
:1036800008050050DC000020B80F0020B00F00201B
:103690009C0F00200C05005030B585B001AD0C2208
:1036A0000649280001F0E0FD0024285D01210134D5
:1036B000FFF732FE0C2CF8D105B030BDC66D00000E
:1036C000F0B53B4C85B0210003220C31684601F077
:1036D000CBFD210009220F3101A801F0C5FDFFF744
:1036E00007FE344B344CC0182368984201D20023A3
:1036F00023602568002D3ED12E006B4604339F5D6C
:1037000001213800FFF708FE01360121380001F0E1
:1037100079F8092EF1D100266B469F5D0121380012
:10372000FFF7FAFD01360021380001F06BF8032E97
:10373000F2D1C82080000138C046C046C046C0460D
:10374000C046C046C046C046C046C046C046C04649
:10375000F1D100210520FFF7DFFD00266B46002197
:10376000985D0136FFF7D8FD032EF7D1FFF7C0FDB6
:103770001330206019E0FFF7BBFD23680025984255
:1037800013D3052000F0CAFE0C4B0D4EC01801D417
:10379000306000E035603068032101F0CDFB00238C
:1037A0000125084A306023601360280005B0F0BD91
:1037B000C66D000010270000980F0020C8FEFFFF14
:1037C000A80F0020A00F002010B50124044001D054
:1037D000441002E00D20FCF717FF200010BD000090
:1037E0007FB5A44E3368002B0BD1A34A1268002A80
:1037F00007D1A24B1B68002B00D139E1FFF760FF16
:1038000036E19F4D2A68002A2AD19C4A1268002A74
:1038100007D0FFF755FF002800D129E1FFF73CFF53
:1038200005E0954A1268002A01D1002BF6D1924B8F
:1038300019681A00002911D03468002C0ED101AD8E
:103840000C22904928001C6001F00EFD285D00212B
:103850000134FFF761FD0C2CF8D109E133681360E6
:1038600000210D2000F0CEFF00210E2000F0CAFF45
:1038700000210F2000F0C6FF2E68012E56D0022E28
:1038800000D19CE0002E00D0ECE0013631007A4CF3
:1038900004202368994300F0B5FF04212368052024
:1038A0000B405942594100F0ADFF1021236806201A
:1038B0000B405942594100F0A5FF802123680901BE
:1038C0000B40594259410C2000F09CFF8021236895
:1038D00009020B40594259410B2000F093FF80210F
:1038E000236849020B40594259410A2000F08AFFDF
:1038F0008021236889020B4059425941092000F078
:1039000081FF80212368C9020B4059425941082098
:1039100000F078FF802321681B030B405942594176
:10392000072000F06FFF31000D2099E00221524C7A
:10393000072023680B405942594100F063FF0820DB
:10394000216801400B005942594100F05BFF802182
:103950002368C9000B4059425941052000F052FF2D
:103960008021236849010B4059425941062000F04B
:1039700049FF80212368C9010B4059425941042065
:1039800000F040FF8021236889030B4059425941D0
:103990000A2000F037FF802321681B040B405942A6
:1039A0005941092000F02EFF31000C2000F02AFFC1
:1039B00031000B2000F026FF31000E2050E02021C6
:1039C0002D4C072023680B405942594100F01AFF43
:1039D0004021236808200B405942594100F012FF52
:1039E0008021236809200B405942594100F00AFF09
:1039F0008021236849000B40594259410A2000F0B8
:103A000001FF8021236889000B40594259410B2056
:103A100000F0F8FE8021236889010B40594259418A
:103A20000C2000F0EFFE8021236849030B4059422F
:103A30005941062000F0E6FE80212368C9030B40AF
:103A400059425941042000F0DDFE802321685B04C7
:103A50000B4059425941052000F0D4FE01210F20AE
:103A600000F0D0FE2B680321581C01F04BFB2960AD
:103A70007FBDC046AC0F0020A40F0020A00F002087
:103A8000B40F0020C66D0000006810B5C30703D551
:103A9000FFF79AFE054B1860054B1B68002B03D0FF
:103AA000024B186800F0CDFA10BDC046AC0F0020E4
:103AB000C00F00200022054B10B51A60044B1B6894
:103AC000934201D000F0BBFA10BDC046AC0F0020FD
:103AD000C00F002070B505000068FFF775FE0400F8
:103AE0006868FFF771FE631E0100042B14D8451EA1
:103AF000042D11D805226A43D318012215009D40D8
:103B00002B00064805682B430360054B1B68002B00
:103B100002D0200000F094FA70BDC046AC0F002027
:103B2000C00F002070B505000068FFF74DFE0400CF
:103B30006868FFF749FE631E0100042B14D8451E78
:103B4000042D11D805226A43D31801229A4013008C
:103B5000064802689A43064B02601B68002B03D09C
:103B60000022200000F06CFA70BDC046AC0F0020AF
:103B7000C00F00202C4BF7B51B680400002B03D1AD
:103B800001204042FFF72CFD01262468344219D061
:103B9000FF226310180212041040FF226112120269
:103BA0000A40DBB210431843204B1B68202B06D180
:103BB000B4401F4BA40EA400E35800021843FFF7C3
:103BC00031FD30E0032525402DD1042C2BD90F23C6
:103BD00022681340062B26D1FF27130901933F04C7
:103BE000019B9D421FDAAB00E3185A68324218D09D
:103BF000531018023840FF21844609025012084031
:103C00006146DBB208431843084B1B68202B06D1E2
:103C10005200920E064B9200D35800021843FFF751
:103C200001FD0135DCE7F7BD9C0F0020DC00002022
:103C3000F46D00000B6810B50200D80701D55810CC
:103C400001E0012040421823012A03DD4A68042ACA
:103C500000D10833024A1360FFF7C2FC10BDC04612
:103C6000DC000020012010B54042FFF7B9FC002025
:103C7000FFF7D8FC10BD00000068F8B5C30702D5F7
:103C8000FFF7A2FD0BE0830726D1042824D90F22D9
:103C900003681A40042A1FD11B091DD000790300B4
:103CA000203B5E2B18D80522002053430B4E9D1855
:103CB000043AAB420CD0052110249F5D3C4200D059
:103CC00080180139520064100029F7D10133F0E760
:103CD00001234000184300E00120F8BDF46E00000D
:103CE000F0B5050085B008680C00FFF76DFD039086
:103CF000022D08DD6068FFF767FD0700A068FFF789
:103D000063FD040001E00124270005236343053B14
:103D10000293012326000193231D9E4234DC3D00C3
:103D20003B1D9D422BDC731E042B23D86B1E042BE2
:103D300020D8029B039A591E019B49191A40204B17
:103D40000AD001228A4019680A431A601D4B0122D9
:103D50001B68002B0ED009E0012088400100186884
:103D600088431860174B1B68002B03D031002800D4
:103D700000F066F9019B01355B000193D0E7029BDF
:103D8000013605330293C7E73D1D042D15D8012CDC
:103D900013D126003300AB40094A11689943094BFF
:103DA00011601B68002B04D0781D0022210000F058
:103DB00047F901340535062CECD105B0F0BDC046FD
:103DC000AC0F0020C00F002010B5034A01210348AA
:103DD000FEF742FD10BDC046D4000020DE6D00009D
:103DE0000120704710B501210D20FFF795FA012140
:103DF0000E20FFF791FA00210F20FFF78DFA044CF7
:103E0000200000F091F91021200000F0A9F910BD68
:103E1000D00F002010B504680D20E30703D564100F
:103E2000FF2C03D91720FCF7EFFB06E0FFF7DAFFC2
:103E3000E1B2024800F0B6F9002010BDD00F00201A
:103E400010B5FFF7CFFF0021034800F0ABF90123C5
:103E50004000184310BDC046D00F002010B5034AE3
:103E600005210348FEF7F8FC10BDC046E000002025
:103E7000CF700000F7B501260468344205D04268CF
:103E8000324202D08368334201D10D2005E0521046
:103E900064100092802C03D91520FCF7B5FB23E0B9
:103EA000009A1620FF2AF8D85B1001931720FF2BE9
:103EB000F3D80E4F0E4D3B68002B03D1280000F0C5
:103EC000F7F93E60E1B2280000F080FA6B46280066
:103ED000197800F0AEF96B462800197900F0A9F9BD
:103EE000280000F0DDFA0020FEBDC046BC0F002017
:103EF000E40F0020F8B5154F05003B680E00144C88
:103F0000002B04D1200000F0D3F901233B60EDB277
:103F10002900200000F05AFAF1B2200000F089F9DF
:103F20000021200000F05EFA002801D040420CE0A1
:103F300001222900200000F044FA200000F06FF96F
:103F40000028FAD0200000F06FF9F8BDBC0F002067
:103F5000E40F002010B501240368234202D0416819
:103F6000214201D10D2004E058104910802803D9C6
:103F70001520FCF749FB07E0FF2901D91620F8E7D7
:103F8000FFF7B8FF4000204310BD10B507211820EF
:103F9000FFF7B0FF7F2801DD0138FF3803007F33D2
:103FA00001DA7F20404264237F215843494200F0D8
:103FB000C3FF012340424000184310BD10B5082143
:103FC0001820FFF797FFC30F181801234010153072
:103FD0004000184310BD10B505211820FFF78AFFD7
:103FE0007F2801DD0138FF3803007F3301DA7F20AD
:103FF000404264237F215843494200F09DFF012342
:104000004000184310BD10B503211820FFF772FFC0
:104010007F2801DD0138FF3803007F3301DA7F207C
:10402000404264237F215843494200F085FF012329
:104030004000184310BD00207047002070477047B3
:104040007047704710B5034A02210348FEF704FC8D
:1040500010BDC04608010020FF70000010B5FFF73A
:1040600045FAC820C000FDF7B7FFFEF767FC04481B
:10407000FEF7B8FDFEF7BEFAFEF720FE10BDC04603
:10408000BD6C000010B5FDF739FF10BD70B50025FF
:1040900004AC24780573A94205D10A4B0A4A2321AE
:1040A0000A4801F061F801600949920052589B00EA
:1040B00002715B588371A3005B58856043710223D2
:1040C000C37170BD577100001A7100006571000066
:1040D000EC710000037B002B04D1437383730361F5
:1040E00001330373704700001FB50191A021002424
:1040F0000068C900D2B24450012A07D0A24203D0BE
:10410000032A05D1042202E0022200E00622134322
:10411000034A8350034B019AC250012343501FBDF1
:10412000540500002405000010B50400FFF7D2FF7D
:10413000A1222368A179D20099506179064A200012
:104140009950217904329950044B19685A689B6838
:10415000FFF7CAFF10BDC0460C050000C40F0020C9
:104160004BB2002B0CDB80233F290CD81F290CD825
:104170000F290CD807290CD803290CD81B060BE0F3
:1041800080239B0408E0DB0406E01B0504E05B05DC
:1041900002E09B0500E0DB050168014A8B50704797
:1041A000240500000368074A99501A00FC32D168C0
:1041B0000029FCD0A321C90058580023C0B2D36005
:1041C0007047C0461C05000007B58022074BD2058A
:1041D0001A6000229A6002321A7111230E32009383
:1041E000034905330348FFF751FF07BDC40F002003
:1041F00000300040D00F0020F8B505000E00170079
:104200000024BC4208D02B68315D1B682800984709
:10421000002801D00134F4E72000F8BD704710B544
:104220001C3000F0D5FB10BD10B51C3000F0C2FBF7
:1042300010BD70B5437E0D00002B05D06430040026
:1042400000F0D5FB002801D0002004E02000290068
:1042500000F0A1FB012070BD10B51C3000F0BEFBCA
:1042600010BD0000F7B50193FA23002504009B0060
:1042700083600D4B4560083303601C300F0016004F
:1042800000F07EFB2000643000F07AFB074AB600A5
:10429000B35827616375019B20009B009B5865768E
:1042A000A576A375FEBDC046CC710000EC71000080
:1042B0000123A022C375837D0C49C133FF33D2058E
:1042C0009B009950437DC133FF339B009950CC2113
:1042D0000369074A490499500521243A9950817D80
:1042E00008329950417D034A995070470C060000EE
:1042F000240500000C050000F7B5050000200C00A7
:10430000019382425CD0161E402E00D940262F0019
:104310001C37380000F04AFBB1222B69D200802103
:104320009C50012289005A50A97E002901D11A62AD
:104330001A600024731E2A69A34206D1019B002B38
:1043400003D0802302219B00D1500123136213006C
:10435000FC33D968002902D1996A0029F9D0996AF9
:1043600000290AD1D960A323DB00D1583800C9B293
:10437000013400F010FBA642DCD8019A2B69002A18
:1043800004D11A00FC32916A00290AD001210022CE
:10439000AA7659611900FC3188680028FCD08A602F
:1043A00007E00121A976D961D16C0029FCD0002158
:1043B000D164FC339A6A002A01D000229A62E0B2EA
:1043C000FEBD10B50123FFF797FF10BD0300AC330E
:1043D00010B504001970643000F0E8FA0123637628
:1043E00010BD0000F8B500220D0001004276AC318E
:1043F000036904000878B121C90058508021890060
:104400005A5001321A629A6026006436300000F079
:10441000DFFA00280ED03000276900F0CBFA1E4BDF
:10442000F8502369FC331A6A002A0CD19A6A002AD0
:10443000F9D008E02369002D0AD11A00FC32916AF4
:10444000002905D10EE09A6A002AF3D11A62DBE74F
:1044500001225A611A00FC3291680029FCD0002127
:10446000916006E00121D961D16C0029FCD00021C6
:10447000D1641A000020FC32916A81420BD00749B6
:1044800090625A5802305A50824204D0043A534241
:1044900053410230C01AF8BD1C050000C4040000DE
:1044A00010B50121FFF79EFF10BD000010B51323CA
:1044B000122202490248FFF7D5FE10BD004000401D
:1044C000E40F002003210A4802680A4302600948F9
:1044D00002680A4302600849084A094B9B1A03DD37
:1044E000043BC858D050FBDC00F0B4F9FBF742FEA7
:1044F00024050040540500407C74000000000020AA
:10450000E4010020FEE7FEE7FEE7FEE7FEE7FEE748
:10451000014B18607047C04620010020F7B500230A
:104520001E2877D83C4B8000C258042A14D006D8E5
:10453000022A0DD00ED80423012A14D069E0062ADD
:104540000ED00BD31A2A0DD002231B2A0BD060E009
:10455000082308E0102306E0202304E0402302E0C3
:10456000802300E001232D4A1268082A04D9092A71
:1045700005D00A21022404E00821002401E01100F2
:104580000124A02501261C272548ED004651254D74
:10459000254E2D681B02AD003D400195234D2D6831
:1045A00000958559AC466746214D3D401D438551D8
:1045B0008359C0259C46009BAD021D40FF236746E2
:1045C0001B023B402B43019D1D43009B5F01602369
:1045D0001F402B003B431C4301238451154C0360B7
:1045E00063680F48002BFBD00024124B01255C6050
:1045F000A123DB00C3584560A025ED0044511BB248
:10460000914207D002D98A1AD34003E0521A93404C
:1046100000E000231800FEBDEC7100002401002022
:10462000007000401C01002004050000180100205B
:10463000FF00FFFFFC700040F0B51E286CD8374B20
:104640008000C258364B1E68002E2ED1C224354839
:10465000A4000759344B03253B40C0273F023B438E
:1046600003518023893C9B00FF3C03512F4F036083
:104670002F4B803CD859FF3CA043D8510437D85920
:10468000A8432043D8510837D8590C35A843083DD2
:104690002843D851A820C0001E508026C120760291
:1046A00080001E501C601E4B1C60002314262148F5
:1046B00034005C43255804006F1C0FD1142058436C
:1046C0002250A0200325C132FF329200C0051550B0
:1046D000194A08001268082A03D10BE0AA4218D12F
:1046E000ECE7082A02D9083AD14002E00820821AF1
:1046F0009140080014225343E3189A680C49513240
:10470000FF32920058605050DA68C1239B00CA50B3
:1047100002E00133032BCBD1F0BDC046EC710000A9
:104720009C10002000E100E0FF00FFFF04050000F6
:104730000090004028010020200100201E4BF0B511
:10474000596C18001D4A002914D0A025A126002369
:104750000124ED05F600D1584F1C06D0D7187F680C
:10476000002F02D027008F40AF5114333C2BF2D1E1
:1047700000234364131DA0254032944600200124E9
:104780000F4EED05DA680F49920057180A49521882
:10479000526C002A0CD01A1F1268511C05D01968DF
:1047A000FF2902D021009140A9513A00FC32506407
:1047B00014339C45E6D1F0BDFC9000402801002058
:1047C0000C0500000090004000B51E2816D80C4AC9
:1047D00083009B58032911D8A0220800C133FF335E
:1047E000D2059B0000F014FB02080406002104E03F
:1047F0000C2102E0042100E00321D15000BDC0469D
:10480000EC7100001E280DD8074B8000C058A02274
:104810000123D2058340002901D1044901E0A121EF
:10482000C90053507047C046EC7100000C050000F1
:10483000030000201E2B0AD8A222A021D200C90505
:104840008858034A9B009B58D84001231840704762
:10485000EC7100002D4B10B51A78012A19D12C4AA1
:104860001268120715D12B4AE0241168F0220800C3
:10487000104021420BD128490968114209D127492A
:10488000274A11608021274A0902116001E030287F
:10489000F1D01A78012A0DD11D490968090709D1FB
:1048A000F0201C4909680140402903D11A490968D0
:1048B000014223D01B68DBB2012B25D1144B1B68AE
:1048C0001B0721D1134B1A68F0231A40A02A04D1E8
:1048D000114A12681A4203D016E0D02A14D1F7E721
:1048E000114B1A68012A03D1C022104B1A600BE049
:1048F0000F4A1A601A68012AFCD1F5E7C12180200D
:10490000C900C0054250D5E710BDC046E00F00F019
:10491000E40F00F0E80F00F0EC0F00F0DFFF07C03D
:1049200004050040186C004000EC064014EC064002
:1049300075930000F7B506000D000C008B1801936D
:10494000019B671B9C4207D0336821781B683000AD
:10495000984701340028F3D13800FEBD70B505003A
:104960000C00081E07D001F0B5F82B6802005B6848
:1049700021002800984770BD10B5FFF7EFFF10BD6C
:1049800010B540220021040000F077FC0023200035
:104990002364636410BD3F23026C10B5541C234094
:1049A000446C9C4201D08154036410BD0023036415
:1049B00043647047436C026C934206D03F21C25C53
:1049C00001330B404364100001E001204042704776
:1049D000036C406C181A00D540307047436C026C71
:1049E000934201D0C05C01E0012040427047036C5B
:1049F000406C5A1C3F231340181A42424241D0B225
:104A000070470120704710B503681322DB6998478F
:104A100010BD70470369054A9950FC331A6A002A91
:104A2000FCD0002201201A627047C0461C0500001D
:104A3000030010B55C331A781F23134001221100C4
:104A400099400D4B0424D967C221036989005C5049
:104A50005A60DA60A0220021D20099500122074951
:104A600052425A50064914305A500C395A500831A3
:104A70005A50FFF79BFF10BD04E100E00C05000059
:104A80001405000010B51430FFF7A2FF10BD10B5DB
:104A90001430FFF7A3FF10BD10B51430FFF78AFFE5
:104AA00010BD0000030070B55E331C780269604BD6
:104AB000D45003005D331C785E4BD4500300613347
:104AC0001C785D4B012C0CD105005F352E78A2259A
:104AD000ED005651050060352E78A125ED005651A8
:104AE00000E00024D4509623DB00994238D9962365
:104AF0001B01994237D996235B01994236D99623F7
:104B00009B01994234D9E1239B01994232D99623E2
:104B1000DB01994231D9E123DB0199422FD9962358
:104B20001B0299422DD9E1231B0299422BD99623CE
:104B30005B02994229D9E1235B02994227D9E123FB
:104B40009B02994225D93D4B994224D9E123DB02AE
:104B5000994223D9E1231B03994221D8384B21E004
:104B60009E23DB021EE09D231B031BE0354B19E057
:104B7000354B17E0EC239B0314E0344B12E0344B2D
:104B800010E0344B0EE0344B0CE0344B0AE0344B75
:104B900008E0344B06E08023DB0403E0324B01E005
:104BA00080235B053149002453500423243953509A
:104BB0001100FC31CC600C62C12101348900146009
:104BC0005C309460535003781F202200D9B2084013
:104BD000824080342648FF345BB20251002B13DA46
:104BE0000F230B40083B234C9B089B001B190324FD
:104BF0002140A140FC348C40DD69A543C0248C4099
:104C000021002943D96111E0194C9B089B001B1915
:104C100003242140A140C025FC348C40AD005E59E6
:104C2000A643C0248C40210031435951026070BD1D
:104C30000C050000140500006C05000090D0030076
:104C400000D0BE0E00B013000050270000A04E00A0
:104C500000F0750000509D0000F0EB0000903A015C
:104C600000E0D70100B0AF0300705F07240500002B
:104C700000E100E000ED00E0F7B5009308AB1B7821
:104C800000250193FA2304009B0083600E4B4560CE
:104C90000833036014300F001600FFF771FE230085
:104CA0005C3327611E70009B084A9B0099582300C3
:104CB0005D331970019B20009B009A5823005E33DE
:104CC000DD701A70FEBDC04668720000EC71000015
:104CD000036910B51A00FC32D2680400002A0AD019
:104CE000A322D20099581430C9B2FFF754FE002213
:104CF0002369FC33DA6010BD10B50248FFF7E8FF06
:104D000010BDC046A01000201D2307B5022200934D
:104D1000024901330248FFF7AFFF07BD0020004002
:104D2000A01000207047000010B500F047F8FFF712
:104D3000F9FF012000F024F8FFF790F9FFF7A2F93E
:104D4000024B002BFAD000E000BFF7E700000000A4
:104D5000084A0949094B10B51B688858FA22190AF4
:104D60001B0618439200002300F0D2F94904C00B3F
:104D7000084310BD0405000000100140041100208C
:104D800070B5041E09D0FFF7E3FF050000F014F82A
:104D9000FFF7DEFF401B8442F8D870BD0022044BB1
:104DA0009A60044A13680133DBB213607047C0464F
:104DB000FC1001400411002070470000C421114A7A
:104DC00089005058104B0340C02000020343535049
:104DD000802391399B02FF39535013608023A32213
:104DE0000021DB05D20099500122A1209A60074BD7
:104DF000C0001950C12002318000195040301950B4
:104E00001A60704700E100E0FF00FFFF0010014062
:104E100002B4714649084900095C49008E4402BC4D
:104E20007047C046002243088B4274D303098B426B
:104E30005FD3030A8B4244D3030B8B4228D3030C6A
:104E40008B420DD3FF22090212BA030C8B4202D30C
:104E50001212090265D0030B8B4219D300E0090A34
:104E6000C30B8B4201D3CB03C01A5241830B8B423D
:104E700001D38B03C01A5241430B8B4201D34B0326
:104E8000C01A5241030B8B4201D30B03C01A52418B
:104E9000C30A8B4201D3CB02C01A5241830A8B4210
:104EA00001D38B02C01A5241430A8B4201D34B02F9
:104EB000C01A5241030A8B4201D30B02C01A52415D
:104EC000CDD2C3098B4201D3CB01C01A5241830911
:104ED0008B4201D38B01C01A524143098B4201D34B
:104EE0004B01C01A524103098B4201D30B01C01A76
:104EF0005241C3088B4201D3CB00C01A52418308F0
:104F00008B4201D38B00C01A524143088B4201D31C
:104F10004B00C01A5241411A00D20146524110467C
:104F20007047FFE701B5002000F0F0F802BDC04671
:104F30000029F7D076E7704703460B437FD4002261
:104F400043088B4274D303098B425FD3030A8B421D
:104F500044D3030B8B4228D3030C8B420DD3FF2287
:104F6000090212BA030C8B4202D31212090265D055
:104F7000030B8B4219D300E0090AC30B8B4201D308
:104F8000CB03C01A5241830B8B4201D38B03C01A4F
:104F90005241430B8B4201D34B03C01A5241030BC6
:104FA0008B4201D30B03C01A5241C30A8B4201D377
:104FB000CB02C01A5241830A8B4201D38B02C01A22
:104FC0005241430A8B4201D34B02C01A5241030A99
:104FD0008B4201D30B02C01A5241CDD2C3098B427E
:104FE00001D3CB01C01A524183098B4201D38B01FB
:104FF000C01A524143098B4201D34B01C01A52419E
:1050000003098B4201D30B01C01A5241C3088B42E2
:1050100001D3CB00C01A524183088B4201D38B00CD
:10502000C01A524143088B4201D34B00C01A52416F
:10503000411A00D201465241104670475DE0CA0F46
:1050400000D04942031000D34042534000229C4606
:1050500003098B422DD3030A8B4212D3FC22890110
:1050600012BA030A8B420CD3890192118B4208D3E6
:10507000890192118B4204D389013AD0921100E048
:105080008909C3098B4201D3CB01C01A524183095C
:105090008B4201D38B01C01A524143098B4201D389
:1050A0004B01C01A524103098B4201D30B01C01AB4
:1050B0005241C3088B4201D3CB00C01A524183082E
:1050C0008B4201D38B00C01A5241D9D243088B4284
:1050D00001D34B00C01A5241411A00D20146634627
:1050E00052415B10104601D34042002B00D549428B
:1050F000704763465B1000D3404201B5002000F0CA
:1051000005F802BD0029F8D016E770477047C04681
:10511000F0B54F464646C0B41604360C99463300E7
:1051200005042C0C070C150C63437E436F43654349
:105130001C0CAD1964199C46A64203D980235B025E
:10514000984647446346250CEF191D044B464A43D5
:1051500043432D0C240464199918C91920000CBC70
:1051600090469946F0BDC0467FB51D000A4B06002B
:105170001B68D868002A02D1084C230001E0130004
:10518000074C0293009133002A000649019400F075
:1051900021F800F023FEC046C4010020546B00003B
:1051A00098720000A5720000084B10B50400002B97
:1051B00002D0002100E000BF054B1868836A002B75
:1051C00000D09847200001F0F3FAC046000000002C
:1051D000D87200000EB403B5010003AB044804CB41
:1051E0000068019300F016F902B008BC03B018473C
:1051F000C40100200E4B70B500251E000D4CE41AB2
:10520000A410A54204D0AB00F35898470135F8E745
:1052100001F0D0FA084B00251E00084CE41AA41037
:10522000A54204D0AB00F35898470135F8E770BDAC
:10523000CC010020CC010020CC010020DC010020AA
:1052400010B5034B0100186800F066F810BDC046A9
:10525000C401002010B5034B0100186800F016F8D7
:1052600010BDC046C4010020002310B59A4203D0EF
:10527000CC5CC4540133F9E710BD0300821893429B
:1052800002D019700133FAE77047000030B50029E9
:105290003ED004390B68002B00DAC9181D4A136888
:1052A0001400002B02D14B60116031E08B420DD90C
:1052B0000A688818834203D118685B6882180A60FC
:1052C0004B60216024E08A4203D813005A68002A08
:1052D000F9D11D685C198C420BD1096869185818FE
:1052E0001960824214D110685268411819605A60DE
:1052F0000EE08C4202D90C23036009E008680C1808
:10530000A24203D114685268201808604A605960AC
:1053100030BDC0460C110020032370B5CD1C9D4349
:10532000083506000C2D01D20C2505E0002D03DA0E
:105330000C230020336040E0A942F9D81F4B1C68C1
:105340001A002100002913D00B685B1B0DD40B2B16
:1053500002D90B60CC181EE08C4202D16368136046
:105360001AE04B6863600C0016E00C004968E9E73E
:10537000134C2368002B03D1300000F033FB206076
:105380002900300000F02EFB431CD1D00323C41CA5
:105390009C43A0420AD12560200007220B30231D28
:1053A0009043C31A09D05A42E25006E0211A300055
:1053B00000F018FB431CEED1BAE770BD0C110020C1
:1053C00008110020936810B5013B9360002B05DAAB
:1053D0009469A34208DBCBB20A2B05D01368581C92
:1053E00010601970C8B201E000F02CFC10BDF8B5D7
:1053F00006000F001400D518AC4208D021783A00FE
:105400003000FFF7DFFF0134431CF5D100E000203E
:10541000F8BD0000F0B59FB006000F0002920593A2
:10542000002804D08369002B01D100F0D3FD7F4B0D
:105430009F4201D1776808E07D4B9F4201D1B76858
:1054400003E07C4B9F4200D1F768BB891B070AD55C
:105450003B69002B07D0002306AD6B6120336B76D0
:105460001033AB763DE03900300000F043FC0028FB
:10547000F1D001204042D6E0059A111D1268059135
:10548000002A00DA7FE00992013423782E2B00D124
:105490008DE021780322684800F082FE002807D0C2
:1054A000654B2A68C01A4023834013432B600134A4
:1054B0002178631C062261480293297600F070FE71
:1054C000002800D19DE05E4B002B00D090E0072229
:1054D000059B07339343083305936B69039A9B1825
:1054E0006B61029C2378002B04D1029BE31A049386
:1054F00012D003E0252BF8D00134F3E7049B029A85
:1055000039003000FFF773FF431C00D186E06A6961
:10551000049B944663446B612378002B7ED0012268
:10552000002352426A6002A95432521801342B609F
:10553000EB60AB601370AB6521780522414800F049
:105540002FFE002808D03F4B2A68C01A0123834051
:1055500013432B600134EFE72B68DA0604D553229E
:10556000202102A8121811701A0704D553222B21EA
:1055700002A81218117022782A2A00D17CE7099B10
:1055800000200A2105E05242EA60022213432B6008
:105590007AE72278303A092A04D84B4301349B1821
:1055A0000120F6E7002800D16FE709936DE76378E3
:1055B0002A2B0AD1059B02341A1D1B680592002B69
:1055C00001DA01235B42079363E700230A201A00F4
:1055D00001346B6021783039092904D84243013401
:1055E00052180123F6E7002B00D152E7079250E74B
:1055F00005AB00933A00144B2900300000E000BFD7
:1056000007E005AB00933A000F4B2900300000F093
:105610008BF80390039B013300D05EE7BB895B06E8
:1056200000D526E70B981FB0F0BDC04610740000EF
:105630003074000050740000E2720000E672000056
:1056400000000000DC720000EF530000F7B5170007
:1056500001938A680B6900900C00934200DA1300F2
:1056600022003B6043321278002A01D001333B60B4
:1056700023689B0602D53B6802333B6006252368FE
:105680001D401ED0230043331B785A1E93412268CD
:1056900092061CD53020E1184331087021005A1CB5
:1056A00045310978A2184332023311700FE022000D
:1056B0000123193201990098089EB047431C0ED06F
:1056C0000135E3683A689B1A9D42F0DBDAE7220075
:1056D000019943320098089DA847431C02D101203C
:1056E000404220E006232068E1683A680340002534
:1056F000042B03D18D1AEB43DB171D40A3682269ED
:10570000934201DD9B1AED180027BD420AD022000A
:1057100001231A3201990098089EB047431CDED03D
:105720000137F2E70020FEBDF0B58BB006920A000B
:1057300043320793059004920A7E0C00109B6E2A58
:1057400000D1ABE011D8632A22D009D8002A00D1B9
:10575000B5E0582A00D0C5E045310A70814A4FE0D3
:10576000642A1DD0692A1BD0BCE0732A00D1AAE0AC
:1057700009D86F2A29D0702A00D0B3E02022096806
:105780000A43226037E0752A1FD0782A33D0A9E077
:105790000E001A684236111D196013683370A4E0B8
:1057A00021681A68080606D4490604D5111D196037
:1057B0000023D55E02E0111D19601568002D3BDA4B
:1057C0002D23049A6D42137036E021681A6808068A
:1057D00006D4490604D51568111D1960ADB202E062
:1057E000111D196015685F4B227E039308276F2AED
:1057F0001DD00A271BE022007821453211705A4A39
:1058000019680392081D226818600D68100602D4FA
:10581000500600D5ADB2D30702D520231A4322602B
:105820001027002D03D1202322689A4322602300F1
:10583000002243331A7002E00A274A4B039363683D
:10584000A360002B09DB0422216891432160002D15
:1058500005D1049E002B11D07BE0002D79D0049E51
:1058600028003900FFF764FB039B013E5B5C2800C6
:1058700033703900FFF7D6FA051EF1D1082F09D190
:105880002368DB0706D563682269934202DC302374
:10589000013E3370049B9B1B23612BE009681A684F
:1058A000080607D4490605D5111D19601368A28A98
:1058B0001A8004E0111D1960136862691A600023E0
:1058C000049E236116E01A68111D196016680021F4
:1058D0006268300000F064FC002801D0801B60602A
:1058E000636803E0260042363270012323610023FF
:1058F000049A1370079B09AA00932100069B059840
:10590000FFF7A4FE431C02D10120404227E0236997
:10591000320006990598079DA847431CF4D02368D8
:1059200000259B070FD4099BE068984217DA1800FE
:1059300015E022000123193206990598079EB04709
:10594000431CE1D00135E368099A9B1A9D42F0DBC4
:10595000E9E72600039B42361B7833708EE70BB0D5
:10596000F0BDC046ED720000FE720000154B10B590
:105970001C68A36B002B15D11820FFF761FC124B9C
:10598000A0630380114B01224380114B8380114B94
:10599000C380114B03810523438106338381002398
:1059A00002614361A46B0D4A206961690C4BFFF7EA
:1059B000AFFB01220023801859412061616148003A
:1059C000400810BDC40100200E330000CDABFFFF26
:1059D000341200006DE6FFFFECDEFFFF2D7F954CDB
:1059E0002DF45158002370B5064C050008002360C3
:1059F00000F0C8FE431C03D12368002B00D02B60AD
:105A000070BDC046E02000200CB430B5164B9DB0F0
:105A10000C1E1D6804DA8B2301202B6040421DE020
:105A2000822302A99B008B810023029008619C4283
:105A300000D0631E8B604B6101235B42CB81209AB7
:105A400021AB2800019300F053FC431C01DA8B23A7
:105A50002B60002C02D00023029A13701DB030BCC2
:105A600008BC02B01847C046C40100200EB410B5EF
:105A70009DB002A9029008610B48822488604861A9
:105A8000012040421FABC881084804CBA400006835
:105A900001938C8100F02CFC0023029A13701DB03E
:105AA00010BC08BC03B01847FFFFFF7FC4010020F3
:105AB00002780B78002A03D0013001319A42F7D0E6
:105AC000D01A7047031C0A7801311A700133002A7A
:105AD000F9D170470023C25C0133002AFBD1581E64
:105AE0007047030030B5002A0DD00C7801335D1EDD
:105AF000013A2C700131002CF5D19A189A4202D04B
:105B00001C700133FAE730BDF0B51E00454B87B07D
:105B10001B680192029308220B00059003911C78E8
:105B200002995D1C09194878104001D02B00F6E756
:105B30002D2C04D19D1C5C780123009304E000907F
:105B40002B2C01D15C789D1C002E02D0102E0AD186
:105B500062E0302C5ED120222B789343582B54D115
:105B600010266C780235009F31007B1E9F412E4B22
:105B7000FF183800FFF7DCF9380004913100FFF717
:105B800051F900230322070094461800029A1219C3
:105B900051780422114201D0303C07E062461140A6
:105BA00017D03722012900D02032A41AA64210DDD6
:105BB0005A1C0BD0B84207D802D1049B9C4203DC8C
:105BC00070430123201801E001235B422C7801354A
:105BD000DCE75A1C0BD10098059A431E9841124BE2
:105BE000C01822231360019B002B0AD117E0009AF2
:105BF000002A00D04042019A002A10D0039A002BBC
:105C000000D06A1E019B1A6009E03024002EAAD140
:105C10000826A8E70A26A6E7302C9CD0A3E707B001
:105C2000F0BDC046C8010020FFFFFF7F10B5130084
:105C30000A00010002480068FFF766FF10BDC04679
:105C4000C4010020F8B505000F001400002804D09E
:105C50008369002B01D100F0BDF9234B9C4201D197
:105C60006C6808E0214B9C4201D1AC6803E0204BFA
:105C70009C4200D1EC68A369A360A3891B070AD5E5
:105C80002369002B07D023682269FEB2981A636942
:105C900098420FDB08E02100280000F02BF80028D4
:105CA000F1D0012040421DE02100280000F024F93D
:105CB0000028F6D1A3680130013BA36023685A1C79
:105CC00022601F706369984205D0A3893000DB070A
:105CD00008D50A2E06D12100280000F00DF9002871
:105CE000DFD13000F8BDC0461074000030740000F1
:105CF00050740000354B70B51D6806000C00002D77
:105D000005D0AB69002B02D1280000F063F9304BBD
:105D10009C4201D16C6808E02E4B9C4201D1AC68DA
:105D200003E02D4B9C4200D1EC68A3899AB2110785
:105D300023D4D10607D4092201203260373213431D
:105D4000A381404240E0530713D5616B002908D07E
:105D500023004433994202D03000FFF797FA002322
:105D600063632422A3899343A3810023636023698F
:105D700023600822A3891343A3812369002B0BD13D
:105D8000A023A2899B00134080229200934203D05B
:105D90002100300000F0B2F90123A289134005D0A0
:105DA0000023A36063695B42A36103E0910700D411
:105DB0006369A36000202369834205D1130603D5DC
:105DC00040231A43A281013870BDC046C40100209F
:105DD00010740000307400005074000010B50620EC
:105DE00000F0AEFB012000F0E3FC0000F7B58A896B
:105DF00005000C0013075AD44B68002B02DC0B6C17
:105E0000002B19DDE76A002F16D000232E682B60C7
:105E100080235B011A4001D0606D14E00123216AE8
:105E20002800B847431C0ED12B68002B0BD01D2B2C
:105E300001D0162B02D12E6000205AE04022A38907
:105E40001343A38155E0A3895B0706D56368C01A95
:105E5000636B002B01D0236CC01A00230200216A5F
:105E60002800E76AB847A389421C06D129681D2982
:105E70003AD8204ACA40D20736D500226260226949
:105E80002260DB0405D5431C02D12B68002B00D116
:105E90006065616B2E600029CED0230044339942A7
:105EA00002D02800FFF7F2F90020606321E00F69BB
:105EB000002FC1D00B680F60DB1B019300239207FA
:105EC00000D14B69A36003E0019B3F181B1A0193AB
:105ED000019B002BB0DD019B3A00216A2800A66AD5
:105EE000B0470028F0DCA389402201201343A3819E
:105EF0004042FEBD010040200B6970B505000C005A
:105F0000002B01D100201CE0002804D08369002B65
:105F100001D100F05FF80B4B9C4201D16C6808E0A6
:105F2000094B9C4201D1AC6803E0084B9C4200D174
:105F3000EC680C22A35E002BE4D021002800FFF7C0
:105F400055FF70BD107400003074000050740000E4
:105F500010B5024900F0B0F810BDC046F95E00006F
:105F6000002310B5040003604360836081814366B1
:105F7000C281036143618361190008225C30FFF72D
:105F80007CF9054B24626362044BA362044BE36219
:105F9000044B236310BDC04681650000A965000065
:105FA000E16500000D66000070B568254B1E5D437D
:105FB0000E0029007431FFF7AFF9041E08D000214C
:105FC0002A00016046600C30A0606832FFF755F986
:105FD000200070BD836913B50400002B28D18364B1
:105FE000C3640365134B144A1B6882620193984291
:105FF00001D101238361200000F020F860602000BF
:1060000000F01CF8A060200000F018F80022E0600A
:1060100004216068FFF7A4FF01220921A068FFF7AF
:106020009FFF02221221E068FFF79AFF0123A3617C
:1060300013BDC046D8720000515F0000F8B51D4B7B
:1060400006001D68AB69002B02D12800FFF7C2FFD4
:106050004835AC686B68013B05D40C22A75E002F65
:1060600010D06834F7E72B68002B01D02D68F0E7DB
:1060700004213000FFF798FF28600028F6D10C2398
:10608000336016E0012320005B42E3810233A381E9
:1060900067662760A760676027616761A7615C30FA
:1060A00008223900FFF7E9F820006763A763A764B7
:1060B000E764F8BDD8720000F7B5040007000026B9
:1060C00001914834002C16D06368A5680093009BAA
:1060D000013B00930DD4AB89012B08D90E22AB5E96
:1060E000013304D029003800019B984706436835E6
:1060F000EDE72468E6E73000FEBD0000F0B58B89CF
:1061000091B006000C009B0726D40E23C95E00291F
:1061100004DA8023A5891D4010D10CE001AA00F00B
:10612000A1FA0028F5DBF023029D1B021D401A4B4B
:10613000ED186B425D418027FF0001E000254027FC
:1061400039003000FFF7E8F800280CD1A3899A0540
:106150001FD402221343A38123004733236023610A
:106160000123636115E080220C4BB362A389206098
:106170001343A38120616761002D0AD00E23E15EE5
:10618000300000F081FA002803D00122A3891343D4
:10619000A38111B0F0BDC04600E0FFFF515F0000D9
:1061A000C9B28218904204D003788B4202D00130E9
:1061B000F8E70020704710B5884202D98B18984242
:1061C00001D3002305E09B1A013A08D3995C81545E
:1061D000FAE7934203D0CC5CC4540133F9E710BD15
:1061E000F8B506000C001500002904D11100FFF7D6
:1061F00093F8040018E0002A03D1FFF747F82C00B9
:1062000012E000F067FA85420ED929003000FFF74E
:1062100083F8071E07D021002A00FFF725F8210088
:106220003000FFF733F83C002000F8BDF0B58E6871
:1062300085B007000C00039201939E4243D890233F
:106240008A89DB001A423ED0032509692368019838
:106250005B1A029363695D43EB0F5D19029B6D103E
:1062600001331B18AB4200D91D00530510D529007E
:106270003800FFF751F8061E14D0029A2169FEF784
:10628000F3FFA289194B134080221343A38112E02C
:106290002A003800FFF7A4FF061E0CD12169380040
:1062A000FEF7F4FF0C23402201203B60A38940420B
:1062B0001343A38117E0029B2661F61826606561EF
:1062C000019EED1AA560019BB34200D21E00320070
:1062D00003992068FFF76FFF0020A3689B1BA36052
:1062E00023689E19266005B0F0BDC0467FFBFFFF06
:1062F000F0B59FB0029005938B890F0016001B0626
:1063000010D50B69002B0DD14021FFF705F838603F
:106310003861002804D10C23029A01381360D8E0B8
:1063200040237B61002306AD6B6120336B76103315
:10633000AB7634002378002B03D1A31B049312D037
:1063400003E0252BF9D00134F4E7A31B3200390018
:106350000298FFF76BFF431C00D1B4E06A69049B0D
:10636000944663446B612378002B00D1ABE001229B
:10637000002352426A6002A95432521801342B6041
:10638000EB60AB601370AB65534E21780522300093
:10639000FFF706FF002807D00123801B83402A68EF
:1063A000013413432B60EFE72B68DA0604D5532240
:1063B000202102A8121811701A0704D553222B218C
:1063C00002A81218117022782A2A03D0099B0020F3
:1063D0000A210EE0059A111D12680591002A01DBC1
:1063E000099204E05242EA60022213432B60013416
:1063F0000BE02278303A092A04D84B4301349B1829
:106400000120F6E7002800D0099323782E2B1ED117
:1064100063782A2B0AD1059B02341A1D1B6805924A
:10642000002B01DA01235B42079310E000230A20CE
:106430001A0001346B6021783039092904D84243AD
:10644000013452180123F6E7002B00D00792234EA7
:10645000217803223000FFF7A3FE002806D0402356
:10646000801B83402A68013413432B602178062265
:106470001B48661C2976FFF793FE002812D0194BA3
:10648000002B06D10722059B07339343083305935E
:1064900014E005AB00933A00134B2900029800E08A
:1064A00000BF07E005AB00933A000F4B29000298AC
:1064B000FFF73AF90390039B013304D06B69039A09
:1064C0009B186B6135E7BB890B985B0601D50120F2
:1064D00040421FB0F0BDC046DC720000E272000016
:1064E000E6720000000000002D62000070B504009C
:1064F0000D1E1F2D04D916230360012040421EE00B
:10650000426C002A04D08B00D2181368002B08D1EB
:10651000200000F031F82A000100200000F01AF8F5
:106520000DE00020012B0AD0591C03D11733236042
:10653000013004E00024280014609847200070BD5A
:1065400010B5034B01001868FFF7D0FF10BDC0461F
:10655000C4010020002370B5064C0500080011009E
:10656000236000F0F7F8431C03D12368002B00D010
:106570002B6070BDE020002010B500F0DBF810BDEE
:1065800070B50C000E25495F00F0B0F8002803DB61
:10659000636D1B18636503E0A289024B1340A3815E
:1065A00070BDC046FFEFFFFFF8B51F008B890500E7
:1065B0000C001600DB0505D50E23C95E0022022360
:1065C00000F074F8A289054B28001340A381320023
:1065D0000E23E15E3B0000F01FF8F8BDFFEFFFFF68
:1065E00070B50C000E25495F00F060F8A389421CCD
:1065F00003D1054A1340A38104E0802252011343D2
:10660000A381606570BDC046FFEFFFFF10B50E238C
:10661000C95E00F015F810BD70B505000800110046
:106620000022064C22601A0000F0BAF8431C03D185
:106630002368002B00D02B6070BDC046E0200020F6
:10664000002370B5064C05000800236000F062F8D6
:10665000431C03D12368002B00D02B6070BDC046C3
:10666000E0200020002370B5064C05000800110052
:10667000236000F057F8431C03D12368002B00D09F
:106680002B6070BDE0200020002370B5064C050093
:106690000800236000F056F8431C03D12368002B48
:1066A00000D02B6070BDC046E020002070B5050012
:1066B000080011000022064C22601A0000F052F877
:1066C000431C03D12368002B00D02B6070BDC04653
:1066D000E02000200B1F1A68101F002A04DA891816
:1066E00004390B68D01804387047000070B50500F5
:1066F000080011000022064C22601A0000F03AF84F
:10670000431C03D12368002B00D02B6070BDC04612
:10671000E020002058220120014B40421A607047BF
:10672000E020002058220120014B40421A607047AF
:10673000E020002058220120014B40421A6070479F
:10674000E02000205822024B00201A607047C0460B
:10675000E020002058220120014B40421A6070477F
:10676000E020002058220120014B40421A6070476F
:10677000E020002058220120014B40421A6070475F
:10678000E0200020044A1368002B03D01818106082
:1067900018007047014BF9E710110020E820002095
:1067A00058220120014B40421A607047E02000202F
:1067B000FEE7C046F8B5C046F8BC08BC9E46704728
:1067C000F8B5C046F8BC08BC9E467047F606000007
:1067D00088060000060700003C070000780700005C
:1067E000B2070000EE070000160800005408000081
:1067F0009A080000F60800003A090000A00900000D
:10680000EC090000140A00004E0A0000980A00007B
:10681000C00A0000F80A0000300B00006C0B0000FA
:10682000F20B0000BA0C0000480D0000A60D00009D
:10683000E80D00000A0E0000120E0000F40E000029
:10684000F6060000F6060000F6060000F606000058
:10685000400F0000AA0F0000141000005E1000009E
:10686000C010000046110000CE1100001C120000F4
:1068700066120000AC120000F81200004413000081
:1068800090130000DE1300003414000072140000A6
:10689000DE1400000E1500005A150000A6150000B9
:1068A000F21500002C16000078160000F606000015
:1068B000F6060000F6060000F6060000C41600000A
:1068C000F416000024170000501700008017000085
:1068D000AC170000F6060000F6060000F606000001
:1068E000F6060000E41700002C18000078180000DD
:1068F000A8180000D4180000021900004C1900006C
:10690000F6060000F6060000F60600007A19000000
:10691000AA190000DA1900000A1A0000361A00004D
:10692000661A0000921A0000BC1A0000E61A000065
:10693000161B0000461B0000881B0000B41B000053
:10694000E41B0000101C0000F6060000F606000024
:10695000F6060000F6060000F6060000401C0000E7
:106960006C1C0000981C0000C41C0000F01C0000FF
:10697000281D0000601D0000981D0000D01D0000B3
:10698000FC1D00002A1E00005A1E0000F606000032
:10699000F6060000F6060000F6060000F606000007
:1069A000F6060000F6060000F6060000F6060000F7
:1069B000F6060000F6060000F6060000F6060000E7
:1069C000F6060000881E0000B61E000066616C73AB
:1069D000650074727565006C697374206F6620259C
:1069E00064206974656D73006F626A656374206FFB
:1069F0006620636C6173733A20256400537461638D
:106A00006B20756E646572666C6F77000D0A564D6B
:106A10002050616E69633A2025730D0A00496E7338
:106A2000756666696369656E74206D656D6F7279F0
:106A300020666F72204D6963726F426C6F636B7377
:106A4000206F626A656374206865617000496E73C7
:106A5000756666696369656E74206D656D6F7279C0
:106A600020666F72204D6963726F426C6F636B7347
:106A700020737461636B00626164206F626A656396
:106A80007420617420256C640A0025783A202564FE
:106A900020776F7264732C20636C61737349442098
:106AA00025640A004865616465723A2025780A0009
:106AB00009307825782C0A00256420256420256477
:106AC0002025640A00426164207265636F7264204D
:106AD000666F756E6420647572696E6720696E6991
:106AE0007469616C697A6174696F6E210A004E6F16
:106AF0007420656E6F75676820726F6F6D206576A4
:106B0000656E20616674657220636F6D7061637479
:106B1000696F6E0A00526573746F72696E67202523
:106B20006420736372697074732E2E2E0053746127
:106B300072746564002D2D2D2D2D0A005065727321
:106B4000697374656E74204D656D6F72792054653C
:106B500073740A0A000A496E697469616C697A691A
:106B60006E67204D656D6F72790A004D656D6F72AD
:106B70007920696E74697469616C697A65643B2017
:106B800077726974696E67207265636F7264732EC1
:106B90002E2E0A005265636F7264206174206F6646
:106BA000667365742025643A2025642025642025B9
:106BB000642025642028256420776F726473290A75
:106BC0000046696E616C3A2063757272656E74205E
:106BD0002564207573656420256420633020256456
:106BE0002063312025640A006E6F6E650072616457
:106BF000696F0064697361626C65526164696F00FA
:106C00006D65737361676552656365697665640078
:106C10007061636B65745265636569766500706168
:106C2000636B657453656E64007265636569766550
:106C300064496E746567657200726563656976653F
:106C4000644D65737361676554797065007265633F
:106C50006569766564537472696E670073656E6406
:106C6000496E74656765720073656E645061697220
:106C70000073656E64537472696E67007365744364
:106C800068616E6E656C0073657447726F75700035
:106C9000736574506F776572007369676E616C53CA
:106CA0007472656E677468004E6F20667265652049
:106CB0007461736B20656E74726965730057656CDF
:106CC000636F6D6520746F204D6963726F426C6FE6
:106CD000636B7321004D656D6F727920636C656124
:106CE0007265642E00416C6C207461736B73207349
:106CF000746F707065640076303533002025732022
:106D000025730000070000000300000043616C6C65
:106D1000696F706500686173546F6E6500706C61B7
:106D200079546F6E6500686173536572766F007396
:106D30006574536572766F00150000000100000055
:106D40000200000004000000050000000600000032
:106D50006E65740068617357694669007374617287
:106D600074576946690073746F7057694669007794
:106D7000696669537461747573006D794950416433
:106D80006472657373007468696E674465736372D7
:106D9000697074696F6E00636C6561725468696EC6
:106DA000674465736372697074696F6E00617070B7
:106DB000656E64546F5468696E6744657363726985
:106DC0007074696F6E000D0E0F04050C0B0A060738
:106DD00008090D0E0F04050C0B0A06070809646963
:106DE00073706C6179006C696768744C6576656C6A
:106DF0000000000000000000010000000200000090
:106E00000300000004000000050000000600000070
:106E10000700000008000000090000000A00000050
:106E20000B0000000C0000000D0000000E00000030
:106E30000F0000001000000012000000140000000D
:106E400016000000180000001A0000001C000000DE
:106E50001E000000200000002300000026000000AB
:106E6000290000002C0000002F000000320000006C
:106E7000360000003A0000003E0000004200000022
:106E8000460000004B0000005000000055000000CC
:106E90005A00000061000000680000006F00000060
:106EA000760000007D000000840000008B000000E0
:106EB0009200000099000000A0000000A700000060
:106EC000AE000000B5000000BC000000C3000000E0
:106ED000CA000000D1000000D8000000DF00000060
:106EE000E6000000ED000000F4000000FB000000E0
:106EF000FF000000000000000008080800080A4A1F
:106F00004000000A5FEA5FEA0ED92ED36E193244C0
:106F100089330C924C924D08080000000488080840
:106F2000040804848488000A448A4000048EC480D3
:106F3000000000048800000EC000000000080001EE
:106F4000224488100C9252524C048C84848E1C82F1
:106F50004C901E1EC244924C06CA525FE21FF01EA5
:106F6000C13E02448ED12E1FE24488100ED12ED194
:106F70002E0ED12EC488000800080000048004886A
:106F80000244880482000EC00EC008048244880EA9
:106F9000D126C0040ED135B36C0C925ED2521C9235
:106FA0005C925C0ED010100E1C9252525C1ED01CD3
:106FB000901E1ED01C90100ED013712E12525ED255
:106FC000521C8808081C1FE242524C12549814921A
:106FD000101010101E113B75B131113935B3710C01
:106FE0009252524C1C925C90100C92524C861C9205
:106FF0005C92510ED00C825C1FE484848412525245
:10700000524C1131312A44113135BB7112524C921C
:1070100052112A4484841EC488101E0EC808080E0B
:1070200010080482410EC242424E048A4000000011
:107030000000001F0804800000000ED2524F101004
:107040001C925C000ED0100E02424ED24E0C925C8E
:10705000900E06C81C88080ED24EC24C10101C920E
:10706000520800080808024002424C10149814927A
:107070000808080806001B75B131001C9252520026
:107080000C92524C001C925C90000ED24EC2000E2C
:10709000D010100006C8049808080EC80700125245
:1070A000524F0011312A4400113135BB00124C8C73
:1070B0009200112A4498001EC4881E06C48C84863F
:1070C000080808080818080C881800000C8360736A
:1070D000656E736F72730074656D7065726174753F
:1070E00072650074696C74580074696C745900742A
:1070F000696C745A00746F756368526561640074DA
:10710000667400656E61626C65446973706C617968
:1071100000736574506978656C00535049436C6125
:1071200073733A3A535049436C617373284E524615
:107130005F5350495F547970652A2C2075696E74CD
:10714000385F742C2075696E74385F742C207569F3
:107150006E74385F742900705F73706920213D2060
:107160004E554C4C002F55736572732F6A6F686EC5
:107170006D616C6F6E65792F4C6962726172792FE7
:1071800041726475696E6F31352F7061636B616731
:1071900065732F73616E646565706D697374727960
:1071A0002F68617264776172652F6E5246352F3099
:1071B0002E362E302F6C69627261726965732F539F
:1071C00050492F5350492E6370700000000000009A
:1071D0000000000033420000F94100001F4200009F
:1071E00029420000594200001D420000000000003A
:1071F0000100000002000000160000000400000072
:107200000500000006000000070000000800000064
:10721000090000000A0000000B0000000C00000044
:107220000D0000000E0000000F0000001A0000001A
:107230001B000000140000001300000011000000FB
:1072400003000000100000001C0000001D000000F2
:107250001E000000120000001500000017000000D2
:1072600018000000190000000000000000000000ED
:10727000154A000035490000854A0000994A00007F
:107280008F4A0000134A0000074A0000A54A000088
:10729000314A0000034A00002C2066756E63746951
:1072A0006F6E3A2000617373657274696F6E20228D
:1072B000257322206661696C65643A2066696C6595
:1072C00020222573222C206C696E6520256425738D
:1072D00025730A004300000064010020232D302B99
:1072E0002000686C4C0065666745464700303132C7
:1072F000333435363738394142434445460030311E
:10730000323334353637383961626364656600007C
:107310002020202020202020202828282828202045
:10732000202020202020202020202020202020205D
:1073300088101010101010101010101010101010D5
:1073400004040404040404040404101010101010B5
:10735000104141414141410101010101010101018E
:1073600001010101010101010101011010101010C2
:10737000104242424242420202020202020202025F
:107380000202020202020202020202101010102087
:1073900000000000000000000000000000000000ED
:1073A00000000000000000000000000000000000DD
:1073B00000000000000000000000000000000000CD
:1073C00000000000000000000000000000000000BD
:1073D00000000000000000000000000000000000AD
:1073E000000000000000000000000000000000009D
:1073F000000000000000000000000000000000008D
:10740000000000000000000000000000000000007C
:10741000000000000000000000000000000000006C
:10742000000000000000000000000000000000005C
:10743000000000000000000000000000000000004C
:10744000000000000000000000000000000000003C
:10745000000000000000000000000000000000002C
:10746000000000000000000000000000000000001C
:047470000000000018
:08747400008DFF7F0100000004
:10747C00FFFFFFFFF36B0000C5260000006C00004F
:10748C00C9260000106C0000CD2600001E6C000008
:10749C00D1260000296C00008D260000396C0000FC
:1074AC00A12600004D6C0000912600005C6C0000D1
:1074BC00D5260000686C0000D9260000716C000015
:1074CC00DD2600007C6C0000E1260000876C0000CB
:1074DC00C1260000906C000089260000996C000009
:1074EC0099260000156D0000AD3200001D6D0000E6
:1074FC00A9320000266D0000B13200002F6D000093
:10750C00B5320000546D0000653500005C6D000064
:10751C0089350000666D0000933500006F6D00002A
:10752C009D3500007A6D0000A7350000866D0000C7
:10753C0073350000976D00007D350000AD6D0000C7
:10754C0069350000E66D0000C93500001800000028
:10755C00D7700000BD3F0000E3700000D73F000073
:10756C00E970000007400000EF7000008B3F000046
:10757C00F5700000E13D0000037100003B4000008D
:10758C0011710000374000000300000002000000F1
:10759C00080000000A000000FFFFFFFF00000000D1
:1075AC00010000000000020001000000FFFFFFFFCF
:1075BC0000000000020000000000040002000000B7
:1075CC00FFFFFFFF000000000300000000000800A8
:1075DC000300000000000000107400003074000074
:1075EC0050740000000000000000000000000000CB
:1075FC0000000000D4720000000000000000000039
:10760C00000000000000000000000000000000006E
:10761C00000000000000000000000000000000005E
:10762C00000000000000000000000000000000004E
:10763C0000000000640100200F73000039010000FD
:10764C00C9410000AD440000094D00000D010000CF
:04765C00000000002A
:04000003000044C5F0
:00000001FF
